:020000040000FA
:04080000F1EF0BF019
:1008100003B276EF05F0F2B494EF05F09EB09CEFD2
:1008200005F09EB2A4EF05F0F2A81AEF04F0F2B2C0
:1008300025EF04F0F2A620EF04F0F2B022EF04F06E
:10084000A0EF0BF0F296F290FF00CD90F2929EA0F6
:100850002FEF04F00101533F2FEF04F0542BAEC1F2
:10086000B2F1AFC1B3F1B0C1B4F1B1C1B5F1AAC138
:10087000AEF1ABC1AFF1ACC1B0F1ADC1B1F1A6C148
:10088000AAF1A7C1ABF1A8C1ACF1A9C1ADF1A2C158
:10089000A6F1A3C1A7F1A4C1A8F1A5C1A9F19EC168
:1008A000A2F19FC1A3F1A0C1A4F1A1C1A5F19AC178
:1008B0009EF19BC19FF19CC1A0F19DC1A1F196C188
:1008C0009AF197C19BF198C19CF199C19DF1CECF4E
:1008D00096F1CFCF97F153C198F154C199F1CF6AF6
:1008E000CE6A0101536B546B9E90CD800FBC0F8E6E
:1008F0000FBA7EEF04F00F8AA0EF0BF00F8C0FBE43
:10090000BAEF04F096C19AF197C19BF198C19CF19E
:1009100099C19DF19AC19EF19BC19FF19CC1A0F12B
:100920009DC1A1F19EC1A2F19FC1A3F1A0C1A4F1FB
:10093000A1C1A5F1A2C1A6F1A3C1A7F1A4C1A8F1CB
:10094000A5C1A9F1A6C1AAF1A7C1ABF1A8C1ACF19B
:10095000A9C1ADF1AAC1AEF1ABC1AFF1ACC1B0F16B
:10096000ADC1B1F1AEC1B2F1AFC1B3F1B0C1B4F13B
:10097000B1C1B5F101015E6B5F6B606B616B96514C
:100980005E2797515F2398516023995161239A51B3
:100990005E279B515F239C5160239D5161239E5193
:1009A0005E279F515F23A0516023A1516123A25173
:1009B0005E27A3515F23A4516023A5516123A65153
:1009C0005E27A7515F23A8516023A9516123AA5133
:1009D0005E27AB515F23AC516023AD516123AE5113
:1009E0005E27AF515F23B0516023B1516123B251F3
:1009F0005E27B3515F23B4516023B5516123D89072
:100A00000101613360335F335E33D890010161339C
:100A100060335F335E33D8900101613360335F33FD
:100A20005E3300C10CF101C10DF102C10EF103C131
:100A30000FF104C110F105C111F106C112F107C196
:100A400013F108C114F109C115F10AC116F10BC166
:100A500017F134C135F111B839EF05F00101620E1B
:100A6000046F010E056F000E066F000E076F42EF58
:100A700005F00101A70E046F020E056F000E066F50
:100A8000000E076F5EC100F15FC101F160C102F1AC
:100A900061C103F19CEC33F003BF04D018BE02D057
:100AA00018A0108C11A05AEF05F010BA5AEF05F0FB
:100AB0000F80108A0CC100F10DC101F10EC102F1CD
:100AC0000FC103F110C104F111C105F112C106F10A
:100AD00013C107F114C108F115C109F116C10AF1DA
:100AE00017C10BF135C134F1A0EF0BF00392ABB29B
:100AF000AB98AB88030103EE00F080517F0BE92631
:100B000004C0EFFF802B8151805D700BD8A48B82D5
:100B100000008051815D700BD8A48B9281518019A7
:100B2000D8B40790A0EF0BF0F2940101453FA0EF7D
:100B30000BF0462BA0EF0BF09E900101533FA0EF6E
:100B40000BF0542BA0EF0BF09E9211B873EF08F04E
:100B5000040062A1ACEF05F08BB4B6EF05F010AC69
:100B6000B6EF05F08B84109CB7EF05F08B9407B4BB
:100B700009EF06F007B009EF06F01EC620F61FC603
:100B800021F61CC61EF61DC61FF61AC61CF61BC68D
:100B90001DF606C608F607C609F604C606F605C61B
:100BA00007F602C604F603C605F626C628F627C6CB
:100BB00029F624C626F625C627F622C624F623C61D
:100BC00025F60EC610F60FC611F60CC60EF60DC6AB
:100BD0000FF60AC60CF60BC60DF62EC630F62FC65B
:100BE00031F62CC62EF62DC62FF62AC62CF62BC6AD
:100BF0002DF616C618F617C619F614C616F615C63B
:100C000017F612C614F613C615F67DEC35F02BEC6C
:100C100035F0077C07AC24EF06F0C274C2B41EEFB7
:100C200006F0C3CFB3F5C4CFB4F50501D890B43303
:100C3000B333D890B433B33325EF06F0C3CF55F1B7
:100C4000C4CF56F125EF06F0C28207B492EF06F04A
:100C500047C14BF148C14CF149C14DF14AC14EF178
:100C60005EC162F15FC163F160C164F161C165F1B0
:100C700096C1B6F197C1B7F198C1B8F199C1B9F170
:100C80009AC1BAF19BC1BBF19CC1BCF19DC1BDF140
:100C90009EC1BEF19FC1BFF1A0C1C0F1A1C1C1F110
:100CA000A2C1C2F1A3C1C3F1A4C1C4F1A5C1C5F1E0
:100CB000A6C1C6F1A7C1C7F1A8C1C8F1A9C1C9F1B0
:100CC000AAC1CAF1ABC1CBF1ACC1CCF1ADC1CDF180
:100CD000AEC1CEF1AFC1CFF1B0C1D0F1B1C1D1F150
:100CE000B2C1D2F1B3C1D3F1B4C1D4F1B5C1D5F120
:100CF000B3C5B5F5B4C5B6F5B5C5B7F5B6C5B8F560
:100D0000010155515B2756515C23E86A5D230E2E85
:100D100092EF06F05CC157F15DC158F15B6B5C6B03
:100D20005D6B078E0201002FA0EF0BF03C0E006FF1
:100D30001950E00BE00AE866128817BE02D017B41B
:100D4000108E00C10CF101C10DF102C10EF103C101
:100D50000FF104C110F105C111F106C112F107C173
:100D600013F108C114F109C115F10AC116F10BC143
:100D700017F134C135F105012F51000AD8B46CEFD9
:100D800007F005012F51010AD8B4F6EF06F005016E
:100D90002F51020AD8B437EF07F005012F51030A8B
:100DA000D8B437EF07F005012F51040AD8B437EF54
:100DB00007F005012F51050AD8B437EF07F00501F8
:100DC0002F51060AD8B437EF07F005012F51070A53
:100DD000D8B437EF07F005012F51320AD8B4F4EF39
:100DE00006F02F6B6CEF07F06CEF07F0050153670F
:100DF00001EF07F0546701EF07F0556701EF07F0C7
:100E0000566705EF07F06CEF07F057C500F158C5BE
:100E100001F159C502F15AC503F10101010E046F38
:100E2000000E056F000E066F000E076F9CEC33F08E
:100E300000C157F501C158F502C159F503C15AF572
:100E400000672AEF07F001672AEF07F002672AEF31
:100E500007F003676CEF07F053C557F554C558F515
:100E600055C559F556C55AF50F886CEF07F00501C1
:100E700030673DEF07F06CEF07F00FBE52EF07F061
:100E800010A057EF07F0010147674EEF07F04867E2
:100E90004EEF07F049674EEF07F04A6752EF07F051
:100EA00057EF07F007AE57EF07F069EF07F00501BE
:100EB000312F6CEF07F03C0E316F302F6CEF07F0E5
:100EC0000101000E626FE00E636FA50E646F010EEC
:100ED000656F0501306B0F880501626B33B772EFE8
:100EE00007F062810CC100F10DC101F10EC102F1E8
:100EF0000FC103F110C104F111C105F112C106F1D6
:100F000013C107F114C108F115C109F116C10AF1A5
:100F100017C10BF135C134F100C10CF101C10DF164
:100F200002C10EF103C10FF104C110F105C111F1AD
:100F300006C112F107C113F108C114F109C115F17D
:100F40000AC116F10BC117F134C135F101018A67ED
:100F5000B1EF07F08B67B1EF07F08C67B1EF07F0E7
:100F60008D67B5EF07F0E5EF07F08EC100F18FC197
:100F700001F190C102F191C103F10101010E046F71
:100F8000000E056F000E066F000E076F9CEC33F02D
:100F900000C18EF101C18FF102C190F103C191F145
:100FA0000067DAEF07F00167DAEF07F00267DAEFC0
:100FB00007F00367E5EF07F08AC18EF18BC18FF16F
:100FC0008CC190F18DC191F10F80D57ED5BE6DD0D1
:100FD000D6CF47F1D7CF48F145C149F1E86AE8CF0C
:100FE0004AF118BE02D018A0108C109047C100F131
:100FF00048C101F149C102F14AC103F101010A0EE0
:10100000046F000E056F000E066F000E076F9CEC5C
:1010100033F003AF1080010154A71BEF08F00F9AC3
:101020000F9C0F9E0101000E5E6F600E5F6F3D0E04
:10103000606F080E616F010147BF2BEF08F0486732
:101040002BEF08F049672BEF08F04A672BEF08F009
:10105000F28850EF08F0F2985E6B5F6B606B616B2B
:10106000966B976B986B996B9A6B9B6B9C6B9D6B5C
:101070009E6B9F6BA06BA16BA26BA36BA46BA56B0C
:10108000A66BA76BA86BA96BAA6BAB6BAC6BAD6BBC
:10109000AE6BAF6BB06BB16BB26BB36BB46BB56B6C
:1010A000D76AD66A0101456B466B0CC100F10DC1D0
:1010B00001F10EC102F10FC103F110C104F111C120
:1010C00005F112C106F113C107F114C108F115C1F0
:1010D00009F116C10AF117C10BF135C134F1A0EFC6
:1010E0000BF0A0EF0BF00201002FB7EF0AF0D59E36
:1010F000D6CF47F1D7CF48F145C149F1E86AE8CFEB
:101100004AF1D76AD66A0101456B466BD58E1950F4
:10111000E00BE00AE866128817BE02D017B4108E02
:1011200016AE1B8C00C10CF101C10DF102C10EF114
:1011300003C10FF104C110F105C111F106C112F193
:1011400007C113F108C114F109C115F10AC116F163
:101150000BC117F134C135F10FA0109A11B8BCEFD3
:1011600008F00101620E046F010E056F000E066F9C
:10117000000E076FC5EF08F00101A70E046F020E05
:10118000056F000E066F000E076F47C100F148C1E2
:1011900001F149C102F14AC103F19CEC33F003BFF4
:1011A000D8EF08F018BE02D018A0108C11B00F8034
:1011B0000CC100F10DC101F10EC102F10FC103F12B
:1011C00010C104F111C105F112C106F113C107F1FB
:1011D00014C108F115C109F116C10AF117C10BF1CB
:1011E00035C134F102013C0E006F00C10CF101C1A8
:1011F0000DF102C10EF103C10FF104C110F105C1DF
:1012000011F106C112F107C113F108C114F109C1AE
:1012100015F10AC116F10BC117F134C135F1050101
:101220002F51000AD8B4C0EF09F005012F51010A6F
:10123000D8B44AEF09F005012F51020AD8B48BEF58
:1012400009F005012F51030AD8B48BEF09F005010D
:101250002F51040AD8B48BEF09F005012F51050A6C
:10126000D8B48BEF09F005012F51060AD8B48BEFE3
:1012700009F005012F51070AD8B48BEF09F00501D9
:101280002F51320AD8B448EF09F02F6BC0EF09F0A4
:10129000C0EF09F00501536755EF09F0546755EFAA
:1012A00009F0556755EF09F0566759EF09F0C0EF9F
:1012B00009F057C500F158C501F159C502F15AC5E9
:1012C00003F10101010E046F000E056F000E066FA1
:1012D000000E076F9CEC33F000C157F501C158F5C3
:1012E00002C159F503C15AF500677EEF09F00167A5
:1012F0007EEF09F002677EEF09F00367C0EF09F0A7
:1013000053C557F554C558F555C559F556C55AF541
:101310000F88C0EF09F00501306791EF09F0C0EFC9
:1013200009F00FBEA6EF09F010A0ABEF09F0010124
:101330004767A2EF09F04867A2EF09F04967A2EFFB
:1013400009F04A67A6EF09F0ABEF09F007AEABEF83
:1013500009F0BDEF09F00501312FC0EF09F03C0E97
:10136000316F302FC0EF09F00101000E626FE00E07
:10137000636FA50E646F010E656F0501306B0F88FA
:101380000501626B33B7C6EF09F062810CC100F151
:101390000DC101F10EC102F10FC103F110C104F141
:1013A00011C105F112C106F113C107F114C108F111
:1013B00015C109F116C10AF117C10BF135C134F19C
:1013C00000C10CF101C10DF102C10EF103C10FF119
:1013D00004C110F105C111F106C112F107C113F1E9
:1013E00008C114F109C115F10AC116F10BC117F1B9
:1013F00034C135F101018A6705EF0AF08B6705EF0B
:101400000AF08C6705EF0AF08D6709EF0AF039EFF3
:101410000AF08EC100F18FC101F190C102F191C1BA
:1014200003F10101010E046F000E056F000E066F3F
:10143000000E076F9CEC33F000C18EF101C18FF1FB
:1014400002C190F103C191F100672EEF0AF001672C
:101450002EEF0AF002672EEF0AF0036739EF0AF069
:101460008AC18EF18BC18FF18CC190F18DC191F148
:101470000F80109047C100F148C101F149C102F14C
:101480004AC103F101010A0E046F000E056F000E40
:10149000066F000E076F9CEC33F003AF1080010164
:1014A00054A75FEF0AF00F9A0F9C0F9E0101000EE8
:1014B0005E6F600E5F6F3D0E606F080E616F47C11B
:1014C00000F148C101F149C102F14AC103F1010132
:1014D000140E046F050E056F000E066F000E076FE9
:1014E0009CEC33F003AF78EF0AF0F2889DEF0AF03E
:1014F000F2985E6B5F6B606B616B966B976B986B32
:10150000996B9A6B9B6B9C6B9D6B9E6B9F6BA06B9F
:10151000A16BA26BA36BA46BA56BA66BA76BA86B4F
:10152000A96BAA6BAB6BAC6BAD6BAE6BAF6BB06BFF
:10153000B16BB26BB36BB46BB56B0CC100F10DC189
:1015400001F10EC102F10FC103F110C104F111C18B
:1015500005F112C106F113C107F114C108F115C15B
:1015600009F116C10AF117C10BF135C134F10400BC
:101570008BB4C2EF0AF010ACC2EF0AF08B84109C5F
:10158000C3EF0AF08B9407B415EF0BF007B015EF1B
:101590000BF01EC620F61FC621F61CC61EF61DC681
:1015A0001FF61AC61CF61BC61DF606C608F607C6A9
:1015B00009F604C606F605C607F602C604F603C613
:1015C00005F626C628F627C629F624C626F625C619
:1015D00027F622C624F623C625F60EC610F60FC639
:1015E00011F60CC60EF60DC60FF60AC60CF60BC6A3
:1015F0000DF62EC630F62FC631F62CC62EF62DC6A9
:101600002FF62AC62CF62BC62DF616C618F617C6C8
:1016100019F614C616F615C617F612C614F613C632
:1016200015F67DEC35F02BEC35F0077C07AC30EF90
:101630000BF0C274C2B42AEF0BF0C3CFB3F5C4CF22
:10164000B4F50501D890B433B333D890B433B33381
:1016500031EF0BF0C3CF55F1C4CF56F131EF0BF0A2
:10166000C28207B49EEF0BF047C14BF148C14CF169
:1016700049C14DF14AC14EF15EC162F15FC163F1F2
:1016800060C164F161C165F196C1B6F197C1B7F16E
:1016900098C1B8F199C1B9F19AC1BAF19BC1BBF136
:1016A0009CC1BCF19DC1BDF19EC1BEF19FC1BFF106
:1016B000A0C1C0F1A1C1C1F1A2C1C2F1A3C1C3F1D6
:1016C000A4C1C4F1A5C1C5F1A6C1C6F1A7C1C7F1A6
:1016D000A8C1C8F1A9C1C9F1AAC1CAF1ABC1CBF176
:1016E000ACC1CCF1ADC1CDF1AEC1CEF1AFC1CFF146
:1016F000B0C1D0F1B1C1D1F1B2C1D2F1B3C1D3F116
:10170000B4C1D4F1B5C1D5F1B3C5B5F5B4C5B6F51D
:10171000B5C5B7F5B6C5B8F5010155515B275651AA
:101720005C23E86A5D230E2E9EEF0BF05CC157F13F
:101730005DC158F15B6B5C6B5D6B078EA0EF0BF0CE
:1017400002C0E0FF005001C0D8FF1000A6B2A6EF13
:101750000BF00CC0A9FF0BC0A8FFA69EA69CA684F8
:10176000F29E550EA76EAA0EA76EA682F28EA694C2
:10177000A6B2B8EF0BF00C2A1200A96EA69EA69C8A
:10178000A680A8500C2A120004012C0E826F35ECA2
:101790000FF097EC34F00C50BDEC0BF0E8CF00F1FB
:1017A0000C50BDEC0BF0E8CF01F101AFDDEF0BF019
:1017B0000101FF0E026FFF0E036F3AEC34F0296750
:1017C000E9EF0BF00401200E826F35EC0FF0EEEF25
:1017D0000BF004012D0E826F35EC0FF064EC32F04B
:1017E0001200076A0F6A106A116A126A0F010D0E61
:1017F000C16E860EC06E030EC26E0F01680E896E3A
:10180000130E926E080E8A6E8A6AF30E936E8B6ABE
:10181000900E946EC80EBDEC0BF0E8CFE8FF109868
:10182000E8A0108810A805D00E0E216E8E0E226E34
:1018300004D00F0E216E8F0E226E35EC36F0F18E35
:10184000F19EFC0EBDEC0BF0E8CF0BF00BA011806D
:101850000BA211820BA411840BA81188C90EBDEC38
:101860000BF0E8CF16F0CA0EBDEC0BF0E8CF17F086
:10187000CB0EBDEC0BF0E8CF18F0CC0EBDEC0BF0AE
:10188000E8CF19F01B6A1C6A0E6A01015B6B5C6B86
:101890005D6B576B586BF29A0101476B486B496B54
:1018A0004A6B4B6B4C6B4D6B4E6B4F6B506B516B74
:1018B000526B456B466BD76AD66A0F01280ED56E00
:1018C000F28A9D90B00ECD6E01015E6B5F6B606B16
:1018D000616B626B636B646B656B666B676B686B8C
:1018E000696B536B546BCF6ACE6A0F9A0F9C0F9E35
:1018F0009D80760ECA6E9D8202013C0E006FCC6AFE
:10190000160EBDEC0BF0E8CF00F1170EBDEC0BF09E
:10191000E8CF01F1180EBDEC0BF0E8CF02F1190E83
:10192000BDEC0BF0E8CF03F1010103AFB2EF0CF017
:1019300097EC34F0160E0C6E00C10BF0A6EC0BF019
:10194000170E0C6E01C10BF0A6EC0BF0180E0C6E0E
:1019500002C10BF0A6EC0BF0190E0C6E03C10BF0DC
:10196000A6EC0BF000C18AF101C18BF102C18CF130
:1019700003C18DF100C18EF101C18FF102C190F15F
:1019800003C191F11A0EBDEC0BF0E8CF00F11B0E74
:10199000BDEC0BF0E8CF01F11C0EBDEC0BF0E8CF75
:1019A00002F11D0EBDEC0BF0E8CF03F1010103AF16
:1019B00008EF0DF097EC34F01A0E0C6E00C10BF02E
:1019C000A6EC0BF01B0E0C6E01C10BF0A6EC0BF09D
:1019D0001C0E0C6E02C10BF0A6EC0BF01D0E0C6E73
:1019E00003C10BF0A6EC0BF01A0EBDEC0BF0E8CF28
:1019F00000F11B0EBDEC0BF0E8CF01F11C0EBDECAD
:101A00000BF0E8CF02F11D0EBDEC0BF0E8CF03F1B7
:101A100000C192F101C193F102C194F103C195F1AA
:101A2000240EAC6E900EAB6E240EAC6E080EB86E2B
:101A3000000EB06E1F0EAF6E0401806B816B0F0144
:101A4000900EAB6E0F019D8A0301806B816BC26BA0
:101A50008B92BDEC3AF0BDEC3AF0880EBDEC0BF089
:101A6000E8CF00F1890EBDEC0BF0E8CF01F10101E8
:101A700001AF53EF0DF097EC34F0880E0C6E00C1FF
:101A80000BF0A6EC0BF0890E0C6E01C10BF0A6EC6E
:101A90000BF0880EBDEC0BF0E8CF00F1890EBDEC29
:101AA0000BF0E8CF01F100C140F601C141F602C1DF
:101AB00042F603C143F615EC3EF09CEC38F0200EE4
:101AC000BDEC0BF0E8CF2FF505012F51FF0AD8A48C
:101AD00071EF0DF02F6B200E0C6E2FC50BF0A6ECE6
:101AE0000BF00501010E306F3C0E316F250EBDEC81
:101AF0000BF0E8CF00F1260EBDEC0BF0E8CF01F1C2
:101B0000270EBDEC0BF0E8CF02F1280EBDEC0BF078
:101B1000E8CF03F1010103AFA8EF0DF097EC34F02B
:101B2000250E0C6E00C10BF0A6EC0BF0260E0C6E11
:101B300001C10BF0A6EC0BF0270E0C6E02C10BF0EE
:101B4000A6EC0BF0280E0C6E03C10BF0A6EC0BF00C
:101B500000C153F501C154F502C155F503C156F555
:101B600000C157F501C158F502C159F503C15AF535
:101B7000290EBDEC0BF0E8CF5BF505015C515B5D18
:101B8000D8A05BC55CF505012F51020A0EE181B8B2
:101B9000D5EF0DF005015C2FD2EF0DF05BC55CF5C4
:101BA000D5EF0DF081BA54EF3EF0210EBDEC0BF0F5
:101BB000E8CF00F1220EBDEC0BF0E8CF01F1230ECF
:101BC000BDEC0BF0E8CF02F1240EBDEC0BF0E8CF3A
:101BD00003F1010103AF1BEF0EF097EC34F0210E7F
:101BE0000C6E00C10BF0A6EC0BF0220E0C6E01C1C6
:101BF0000BF0A6EC0BF0230E0C6E02C10BF0A6EC62
:101C00000BF0240E0C6E03C10BF0A6EC0BF0210EB2
:101C1000BDEC0BF0E8CF00F1220EBDEC0BF0E8CFED
:101C200001F1230EBDEC0BF0E8CF02F1240EBDEC68
:101C30000BF0E8CF03F100C15DF501C15EF502C113
:101C40005FF503C160F5E4EC37F0E6EC36F03EEC0E
:101C500036F005012F51030A12E005012F51040A45
:101C60001DE005012F51050A24E005012F51060A48
:101C700032E005012F51070A38E07EEF0EF0ACC5C7
:101C800000F101010F0E001701010051000A36E0BA
:101C900001010051050A32E07BEF0EF0ACC500F106
:101CA00001010F0E001701010051000A27E07BEF30
:101CB0000EF00501AC51000A21E00501AC51150AF6
:101CC0001DE00501AC51300A19E00501AC51450A8F
:101CD00015E07BEF0EF00501AC51000A0FE00501A5
:101CE000AC51300A0BE07BEF0EF00501AC51000A5D
:101CF00005E07BEF0EF081BA54EF3EF0CFEC35F00B
:101D000007900001F28EF28C07B0FBEF2FF00FB0BE
:101D100097EF29F010BE97EF29F012B897EF29F04E
:101D20000FB836EF23F00301805181197F0BD8B42F
:101D3000FBEF2FF013EE00F081517F0BE126812B9A
:101D4000E7CFE8FFE00BD8B4FBEF2FF023EE82F0F3
:101D5000C2513F0BD926E7CFDFFFC22BDF50780AF5
:101D6000D8A4FBEF2FF007808EC100F18FC101F1E5
:101D700090C102F191C103F10101040E046F000E44
:101D8000056F000E066F000E076F9CEC33F000AF7E
:101D9000D3EF0EF00101030E8E6F000E8F6F000E59
:101DA000906F000E916F03018251720AD8B47EEFDA
:101DB00029F08251520AD8B47EEF29F08251750A77
:101DC000D8B47EEF29F08251630AD8B4B5EF2CF075
:101DD0008251690AD8B42DEF26F082517A0AD8B41C
:101DE00040EF27F08251490AD8B4CCEF25F0825158
:101DF000500AD8B4EAEF24F08251700AD8B42DEF1B
:101E000025F08251540AD8B458EF25F08251740A53
:101E1000D8B49EEF25F08251410AD8B449EF0FF0B3
:101E200082516D0AD8B453EF13F082514D0AD8B4E1
:101E30006CEF13F08251730AD8B4AEEF28F08251E0
:101E4000530AD8B413EF29F082514C0AD8B4CFEF1B
:101E50001AF08251760AD8B4FBEF13F08251590A76
:101E6000D8B4A4EF12F0ECEF2CF0040114EE00F063
:101E700080517F0BE12682C4E7FF802B1200040112
:101E80000D0E826F35EC0FF00A0E826F35EC0FF0FD
:101E900012000401410E826F35EC0FF003018351F3
:101EA000310AD8B4C4EF11F003018351320AD8B417
:101EB000F4EF10F003018351330AD8B47DEF10F032
:101EC00003018351340AD8B46DEF0FF004013F0EC3
:101ED000826F35EC0FF0EAEF2CF0CC0EBDEC0BF07E
:101EE000E8CF0BF004012C0E826F35EC0FF00301EC
:101EF0008451310AD8B491EF0FF003018451300AB4
:101F0000D8B493EF0FF0030184514D0AD8B49DEF7C
:101F10000FF003018451540AD8B4A4EF0FF0BBEFC3
:101F20000FF08A8401D08A940BAE04D00BAC02D09F
:101F30000BBA21D0E00E0B1218D01F0E0B168539EC
:101F4000E844E00B0B1211D0E00E0B16D8EC34F085
:101F500085C332F186C333F10101296BE5EC34F01E
:101F60005CEC34F000511F0B0B12CC0E0C6E0BC04E
:101F70000BF0A6EC0BF00401340E826F35EC0FF081
:101F800004012C0E826F35EC0FF0CC0EBDEC0BF083
:101F9000E8CF19F08AB406D00401300E826F35EC18
:101FA0000FF005D00401310E826F35EC0FF0040103
:101FB0002C0E826F35EC0FF01938E840070BE8CF94
:101FC00082F40401300E822735EC0FF004012C0E50
:101FD000826F35EC0FF097EC34F019501F0BE8CFFF
:101FE00000F13AEC34F032C182F40401300E822761
:101FF00035EC0FF033C182F40401300E822735EC4A
:102000000FF004012C0E826F35EC0FF097EC34F0DA
:102010002CC000F100AF0BD0FF0E016FFF0E026F5E
:10202000FF0E036F04012D0E826F35EC0FF03AECBA
:1020300034F031C182F40401300E822735EC0FF008
:1020400032C182F40401300E822735EC0FF033C127
:1020500082F40401300E822735EC0FF004012C0EBF
:10206000826F35EC0FF097EC34F02BC000F13AECB6
:1020700034F031C182F40401300E822735EC0FF0C8
:1020800032C182F40401300E822735EC0FF033C1E7
:1020900082F40401300E822735EC0FF004012C0E7F
:1020A000826F35EC0FF097EC34F02DC000F100AFEB
:1020B0000BD0FF0E016FFF0E026FFF0E036F0401C6
:1020C0002D0E826F35EC0FF03AEC34F031C182F412
:1020D0000401300E822735EC0FF032C182F4040186
:1020E000300E822735EC0FF033C182F40401300E3C
:1020F000822735EC0FF0EAEF2CF0CB0EBDEC0BF0A5
:10210000E8CF0BF004012C0E826F35EC0FF00301C9
:102110008451450AD8B4A1EF10F003018451440A58
:10212000D8B4A4EF10F003018451300AD8B4A7EF5B
:1021300010F003018451310AD8B4ABEF10F0B6EFC0
:1021400010F00B9EB0EF10F00B8EB0EF10F0FC0E05
:102150000B16B0EF10F0FC0E0B160B80B0EF10F06A
:10216000CB0E0C6E0BC00BF0A6EC0BF00401330E83
:10217000826F35EC0FF004012C0E826F35EC0FF0FE
:10218000CB0EBDEC0BF0E8CF18F018BECFEF10F07F
:102190000401450E826F35EC0FF0D4EF10F004010E
:1021A000440E826F35EC0FF004012C0E826F35EC7B
:1021B0000FF00401300E826F35EC0FF004012C0E8D
:1021C000826F35EC0FF018B0EDEF10F00401300E17
:1021D000826F35EC0FF0F2EF10F00401310E826FD8
:1021E00035EC0FF0EAEF2CF0CA0EBDEC0BF0E8CFA7
:1021F0000BF004012C0E826F35EC0FF003018451BB
:10220000450AD8B430EF11F003018451440AD8B420
:1022100033EF11F0030184514D0AD8B43CEF11F0B3
:1022200003018451410AD8B436EF11F003018451FF
:10223000460AD8B439EF11F003018451560AD8B4D4
:1022400044EF11F003018451500AD8B44FEF11F05C
:1022500003018451520AD8B452EF11F05BEF11F030
:102260000B9E55EF11F00B8E55EF11F00B9C55EFB7
:1022700011F00B8C55EF11F0FC0E0B1685C3E8FF27
:10228000030B0B1255EF11F0C70E0B1685C3E8FFB9
:10229000070BE846E846E8460B1255EF11F00B84B1
:1022A00055EF11F00B9455EF11F0CA0E0C6E0BC0E8
:1022B0000BF0A6EC0BF0CA0EBDEC0BF0E8CF17F05C
:1022C0000401320E826F35EC0FF004012C0E826F88
:1022D00035EC0FF017BE74EF11F00401450E826F5C
:1022E00035EC0FF079EF11F00401440E826F35ECFC
:1022F0000FF004012C0E826F35EC0FF017C0E8FFD1
:10230000030BE8CF82F40401300E822735EC0FF086
:1023100004012C0E826F35EC0FF017BC97EF11F013
:102320000401410E826F35EC0FF09CEF11F00401B7
:10233000460E826F35EC0FF004012C0E826F35ECE7
:102340000FF017C0E8FF380BE842E842E842E8CF58
:1023500082F40401300E822735EC0FF004012C0EBC
:10236000826F35EC0FF017B4BDEF11F00401520E7F
:10237000826F35EC0FF0C2EF11F00401500E826F46
:1023800035EC0FF0EAEF2CF0C90EBDEC0BF0E8CF06
:102390000BF004012C0E826F35EC0FF00301845119
:1023A000450AD8B4E2EF11F003018451440AD8B4CD
:1023B000E5EF11F0030184514D0AD8B4E8EF11F0B4
:1023C000F6EF11F00B9EF0EF11F00B8EF0EF11F025
:1023D000F80E0B1685C3E8FF070B0B12F0EF11F098
:1023E000C90E0C6E0BC00BF0A6EC0BF00401310E05
:1023F000826F35EC0FF004012C0E826F35EC0FF07C
:10240000C90EBDEC0BF0E8CF16F016BE06D00401E5
:10241000450E826F35EC0FF005D00401440E826F3B
:1024200035EC0FF004012C0E826F35EC0FF016C066
:10243000E8FF070BE8CF82F40401300E822735EC69
:102440000FF004012C0E826F35EC0FF0078097EC33
:1024500034F027C0E8FF003B00430043030B3AEC95
:1024600034F033C182F40401300E822735EC0FF0D2
:1024700004012C0E826F35EC0FF097EC34F027C07E
:1024800001F1019F019D28C000F101013AEC34F0F7
:102490002FC182F40401300E822735EC0FF030C1D9
:1024A00082F40401300E822735EC0FF031C182F442
:1024B0000401300E822735EC0FF032C182F40401A2
:1024C000300E822735EC0FF033C182F40401300E58
:1024D000822735EC0FF004012C0E826F35EC0FF0E3
:1024E00097EC34F029C001F12AC000F1D8900133F3
:1024F0000033D8900133003301013AEC34F02FC19E
:1025000082F40401300E822735EC0FF030C182F4E2
:102510000401300E822735EC0FF031C182F4040142
:10252000300E822735EC0FF032C182F40401300EF8
:10253000822735EC0FF033C182F40401300E82277C
:1025400035EC0FF0EAEF2CF0FC0EBDEC0BF0E8CF11
:102550000BF003018351520AD8B4DBEF12F00301F0
:102560008351720AD8B4DEEF12F003018351500A8E
:10257000D8B4E1EF12F003018351700AD8B4E4EF4C
:1025800012F003018351550AD8B4E7EF12F00301AA
:102590008351750AD8B4EAEF12F003018351430A5C
:1025A000D8B4F3EF12F003018351630AD8B4F6EF05
:1025B00012F0FFEF12F00B90F9EF12F00B80F9EF31
:1025C00012F00B92F9EF12F00B82F9EF12F00B946C
:1025D000F9EF12F00B84F9EF12F00B96F9EF12F00D
:1025E0000B86F9EF12F00B98F9EF12F00B88F9EF68
:1025F00012F0FC0E0C6E0BC00BF0A6EC0BF00401FD
:10260000590E826F35EC0FF01190119211941198C0
:10261000FC0EBDEC0BF0E8CF0BF00BA011800BA271
:1026200011820BA411840BA8118811A01FEF13F0C5
:102630000401520E826F35EC0FF024EF13F0040109
:10264000720E826F35EC0FF011A82EEF13F004011B
:10265000430E826F35EC0FF033EF13F00401630E7D
:10266000826F35EC0FF011A23DEF13F00401500E14
:10267000826F35EC0FF042EF13F00401700E826FA1
:1026800035EC0FF011A44CEF13F00401550E826FDE
:1026900035EC0FF051EF13F00401750E826F35EC3D
:1026A0000FF0EAEF2CF004016D0E826F35EC0FF0A5
:1026B00003018351300AD8B4ABEF13F00301835107
:1026C000310AD8B4BEEF13F003018351320AD8B4F3
:1026D000D1EF13F0ECEF2CF004014D0E826F35ECCE
:1026E0000FF0D8EC34F084C331F185C332F186C3E6
:1026F00033F10101296BE5EC34F05CEC34F00301BB
:102700008351300AD8B493EF13F003018351310A97
:10271000D8B49BEF13F003018351320AD8B4A3EF6E
:1027200013F0ECEF2CF0FD0E0C6E00C10BF0A6ECDC
:102730000BF0ABEF13F0FE0E0C6E00C10BF0A6EC2D
:102740000BF0BEEF13F0FF0E0C6E00C10BF0A6EC09
:102750000BF0D1EF13F00401300E826F35EC0FF067
:1027600004012C0E826F35EC0FF097EC34F0FD0E67
:10277000BDEC0BF0E8CF00F1E2EF13F00401310EF5
:10278000826F35EC0FF004012C0E826F35EC0FF0E8
:1027900097EC34F0FE0EBDEC0BF0E8CF00F1E2EF69
:1027A00013F00401320E826F35EC0FF097EC34F029
:1027B00004012C0E826F35EC0FF0FF0EBDEC0BF018
:1027C000E8CF00F13AEC34F031C182F40401300E6C
:1027D000822735EC0FF032C182F40401300E8227DB
:1027E00035EC0FF033C182F40401300E822735EC52
:1027F0000FF0EAEF2CF003018351300AD8B4A0EFB8
:1028000015F003018351310AD8B4D7EF15F0030155
:102810008351320AD8B48CEF17F003018351330A85
:10282000D8B441EF19F003018351340AD8B4E7EF6B
:1028300019F003018351730AD8B482EF14F0030135
:102840008351760AD8B484EF14F003018351740ADB
:10285000D8B46FEF14F003018351540AD8B434EFA5
:1028600014F0D8A4ECEF2CF00401760E826F35EC56
:102870000FF00401540E826F35EC0FF00784000155
:10288000880E0C6ED8EC34F02981030184512D0A96
:10289000D8B44DEF14F00101299185C32FF186C3FF
:1028A00030F187C331F188C332F189C333F1E5ECEC
:1028B00034F05CEC34F000C10BF0A6EC0BF001C17D
:1028C0000BF0A6EC0BF0880EBDEC0BF0E8CF40F659
:1028D000890EBDEC0BF0E8CF41F67AEF14F004015D
:1028E000760E826F35EC0FF00401740E826F35ECBA
:1028F0000FF007840001880E0C6EC4EC0BF00794F7
:1029000097EF23F082EC14F00401760E826F35EC21
:102910000FF00401760E826F35EC0FF0078414EC93
:1029200031F004012C0E826F35EC0FF00101036BC6
:10293000026B3BC601F13AC600F101AFA5EF14F0FE
:102940000101FF0E026FFF0E036F3AEC34F02967AE
:10295000ACEF14F0B1EF14F004012D0E826F35ECE2
:102960000FF02FC182F40401300E822735EC0FF0F6
:1029700030C182F40401300E822735EC0FF031C1F2
:1029800082F40401300E822735EC0FF032C182F45C
:102990000401300E822735EC0FF033C182F40401BC
:1029A000300E822735EC0FF004012C0E826F35ECCF
:1029B0000FF00101036B026B3DC601F13CC600F153
:1029C00001AFE8EF14F00101FF0E026FFF0E036F7D
:1029D0003AEC34F02967EFEF14F0F4EF14F004014F
:1029E0002D0E826F35EC0FF02FC182F40401300EF2
:1029F000822735EC0FF030C182F40401300E8227BB
:102A000035EC0FF031C182F40401300E822735EC31
:102A10000FF032C182F40401300E822735EC0FF042
:102A200033C182F40401300E822735EC0FF004012B
:102A30002C0E826F35EC0FF00101036B026B3FC669
:102A400001F13EC600F101AF2BEF15F00101FF0EC1
:102A5000026FFF0E036F3AEC34F0296732EF15F086
:102A600037EF15F004012D0E826F35EC0FF02FC1FA
:102A700082F40401300E822735EC0FF030C182F46D
:102A80000401300E822735EC0FF031C182F40401CD
:102A9000300E822735EC0FF032C182F40401300E83
:102AA000822735EC0FF033C182F40401300E822707
:102AB00035EC0FF004012C0E826F35EC0FF00101A4
:102AC000036B026B37C601F136C600F101AF6EEF42
:102AD00015F00101FF0E026FFF0E036F3AEC34F0A8
:102AE000296775EF15F07AEF15F004012D0E826F4E
:102AF00035EC0FF02FC182F40401300E822735EC43
:102B00000FF030C182F40401300E822735EC0FF053
:102B100031C182F40401300E822735EC0FF032C14E
:102B200082F40401300E822735EC0FF033C182F4B9
:102B30000401300E822735EC0FF0079497EF23F055
:102B40000401760E826F35EC0FF00401300E826FB7
:102B500035EC0FF004012C0E826F35EC0FF005EC14
:102B600035F097EC34F000C600F101C601F13AEC03
:102B700034F030C182F40401300E822735EC0FF0BE
:102B800031C182F40401300E822735EC0FF032C1DE
:102B900082F40401300E822735EC0FF033C182F449
:102BA0000401300E822735EC0FF097EF23F004017B
:102BB000760E826F35EC0FF00401310E826F35EC2A
:102BC0000FF007840101036B026B02C600F103C61C
:102BD00001F101AFF0EF15F0FF0E026FFF0E036F72
:102BE0000101076B066B04C604F105C605F105AFCC
:102BF000FEEF15F0FF0E066FFF0E076FA1EC33F02E
:102C00000101076B066B06C604F107C605F105AFA7
:102C10000EEF16F0FF0E066FFF0E076FA1EC33F0FC
:102C20000101076B066B08C604F109C605F105AF83
:102C30001EEF16F0FF0E066FFF0E076FA1EC33F0CC
:102C4000D89001010333023301330033D8900101DE
:102C5000033302330133003304012C0E826F35EC51
:102C60000FF00101036B026B01C101F100C100F122
:102C700001AF40EF16F00101FF0E026FFF0E036F70
:102C80003AEC34F0296747EF16F04CEF16F00401E8
:102C90002D0E826F35EC0FF02FC182F40401300E3F
:102CA000822735EC0FF030C182F40401300E822708
:102CB00035EC0FF031C182F40401300E822735EC7F
:102CC0000FF032C182F40401300E822735EC0FF090
:102CD00033C182F40401300E822735EC0FF001017C
:102CE000036B026B0AC600F10BC601F101AF7DEF69
:102CF00016F0FF0E026FFF0E036F0101076B066BEC
:102D00000CC604F10DC605F105AF8BEF16F0FF0EF2
:102D1000066FFF0E076FA1EC33F00101076B066B26
:102D20000EC604F10FC605F105AF9BEF16F0FF0EBE
:102D3000066FFF0E076FA1EC33F00101076B066B06
:102D400010C604F111C605F105AFABEF16F0FF0E8A
:102D5000066FFF0E076FA1EC33F0D890010103332B
:102D6000023301330033D8900101033302330133BE
:102D7000003304012C0E826F35EC0FF00101036B60
:102D8000026B01C101F100C100F101AFCDEF16F0FE
:102D90000101FF0E026FFF0E036F3AEC34F029675A
:102DA000D4EF16F0D9EF16F004012D0E826F35EC3A
:102DB0000FF02FC182F40401300E822735EC0FF0A2
:102DC00030C182F40401300E822735EC0FF031C19E
:102DD00082F40401300E822735EC0FF032C182F408
:102DE0000401300E822735EC0FF033C182F4040168
:102DF000300E822735EC0FF00101036B026B12C617
:102E000000F113C601F101AF0AEF17F0FF0E026FD8
:102E1000FF0E036F0101076B066B14C604F115C6A4
:102E200005F105AF18EF17F0FF0E066FFF0E076FE5
:102E3000A1EC33F00101076B066B16C604F117C64F
:102E400005F105AF28EF17F0FF0E066FFF0E076FB5
:102E5000A1EC33F00101076B066B18C604F119C62B
:102E600005F105AF38EF17F0FF0E066FFF0E076F85
:102E7000A1EC33F0D8900101033302330133003366
:102E8000D8900101033302330133003304012C0EC7
:102E9000826F35EC0FF00101036B026B01C101F190
:102EA00000C100F101AF5AEF17F00101FF0E026FF0
:102EB000FF0E036F3AEC34F0296761EF17F066EF0D
:102EC00017F004012D0E826F35EC0FF02FC182F444
:102ED0000401300E822735EC0FF030C182F404017A
:102EE000300E822735EC0FF031C182F40401300E30
:102EF000822735EC0FF032C182F40401300E8227B4
:102F000035EC0FF033C182F40401300E822735EC2A
:102F10000FF0079497EF23F00401760E826F35ECE3
:102F20000FF00401320E826F35EC0FF007840101BF
:102F3000036B026B1AC600F11BC601F101AFA5EFCE
:102F400017F0FF0E026FFF0E036F0101076B066B98
:102F50001CC604F11DC605F105AFB3EF17F0FF0E57
:102F6000066FFF0E076FA1EC33F00101076B066BD4
:102F70001EC604F11FC605F105AFC3EF17F0FF0E23
:102F8000066FFF0E076FA1EC33F00101076B066BB4
:102F900020C604F121C605F105AFD3EF17F0FF0EEF
:102FA000066FFF0E076FA1EC33F0D89001010333D9
:102FB000023301330033D89001010333023301336C
:102FC000003304012C0E826F35EC0FF00101036B0E
:102FD000026B01C101F100C100F101AFF5EF17F083
:102FE0000101FF0E026FFF0E036F3AEC34F0296708
:102FF000FCEF17F001EF18F004012D0E826F35EC95
:103000000FF02FC182F40401300E822735EC0FF04F
:1030100030C182F40401300E822735EC0FF031C14B
:1030200082F40401300E822735EC0FF032C182F4B5
:103030000401300E822735EC0FF033C182F4040115
:10304000300E822735EC0FF00101036B026B22C6B4
:1030500000F123C601F101AF32EF18F0FF0E026F4D
:10306000FF0E036F0101076B066B24C604F125C632
:1030700005F105AF40EF18F0FF0E066FFF0E076F6A
:10308000A1EC33F00101076B066B26C604F127C6DD
:1030900005F105AF50EF18F0FF0E066FFF0E076F3A
:1030A000A1EC33F00101076B066B28C604F129C6B9
:1030B00005F105AF60EF18F0FF0E066FFF0E076F0A
:1030C000A1EC33F0D8900101033302330133003314
:1030D000D8900101033302330133003304012C0E75
:1030E000826F35EC0FF00101036B026B01C101F13E
:1030F00000C100F101AF82EF18F00101FF0E026F75
:10310000FF0E036F3AEC34F0296789EF18F08EEF69
:1031100018F004012D0E826F35EC0FF02FC182F4F0
:103120000401300E822735EC0FF030C182F4040127
:10313000300E822735EC0FF031C182F40401300EDD
:10314000822735EC0FF032C182F40401300E822761
:1031500035EC0FF033C182F40401300E822735ECD8
:103160000FF00101036B026B2AC600F12BC601F1BF
:1031700001AFBFEF18F0FF0E026FFF0E036F0101EA
:10318000076B066B2CC604F12DC605F105AFCDEF1C
:1031900018F0FF0E066FFF0E076FA1EC33F0010170
:1031A000076B066B2EC604F12FC605F105AFDDEFE8
:1031B00018F0FF0E066FFF0E076FA1EC33F0010150
:1031C000076B066B30C604F131C605F105AFEDEFB4
:1031D00018F0FF0E066FFF0E076FA1EC33F0D890CA
:1031E00001010333023301330033D890010103336B
:1031F00002330133003304012C0E826F35EC0FF0E3
:103200000101036B026B01C101F100C100F101AFCB
:103210000FEF19F00101FF0E026FFF0E036F3AEC82
:1032200034F0296716EF19F01BEF19F004012D0E89
:10323000826F35EC0FF02FC182F40401300E82272B
:1032400035EC0FF030C182F40401300E822735ECEA
:103250000FF031C182F40401300E822735EC0FF0FB
:1032600032C182F40401300E822735EC0FF033C1F5
:1032700082F40401300E822735EC0FF0079497EFAB
:1032800023F00401760E826F35EC0FF00401330E4B
:10329000826F35EC0FF004012C0E826F35EC0FF0CD
:1032A00085C382F435EC0FF0640E0D6E0301855179
:1032B000320A02E16A0E0D6E03018551330A02E102
:1032C000700E0D6E03018551340A02E1760E0D6E0B
:1032D00003018551350A02E17C0E0D6E0301855113
:1032E000360A02E1820E0D6E03018651780A65E00E
:1032F0000DC00CF0D8EC34F02981030187512D0A60
:10330000D8B485EF19F00101299188C32FF189C341
:1033100030F18AC331F18BC332F18CC333F1E5EC68
:1033200034F05CEC34F000C10BF0A6EC0BF001C102
:103330000BF0A6EC0BF0D8EC34F0298103018E5190
:103340002D0AD8B4A6EF19F0010129918FC32FF1EE
:1033500090C330F191C331F192C332F193C333F191
:10336000E5EC34F05CEC34F000C10BF0A6EC0BF0B3
:1033700001C10BF0A6EC0BF0D8EC34F0298103016D
:1033800095512D0AD8B4C7EF19F00101299196C3C0
:103390002FF197C330F198C331F199C332F19AC339
:1033A00033F1E5EC34F05CEC34F000C10BF0A6EC4A
:1033B0000BF001C10BF0A6EC0BF00DC00CF0C4EC4F
:1033C0000BF0C4EC0BF0C4EC0BF097EF23F004010E
:1033D000760E826F35EC0FF00401340E826F35ECFF
:1033E0000FF003018451780AD8B4BFEF1AF03E0EF3
:1033F0000C6ED8EC34F02981030185512D0AD8B424
:1034000004EF1AF00101299186C32FF187C330F12F
:1034100088C331F189C332F18AC333F1E5EC34F06A
:103420005CEC34F000C10BF0A6EC0BF001C10BF02A
:10343000A6EC0BF0D8EC34F0298103018C512D0A55
:10344000D8B425EF1AF0010129918DC32FF18EC355
:1034500030F18FC331F190C332F191C333F1E5EC18
:1034600034F05CEC34F000C10BF0A6EC0BF001C1C1
:103470000BF0A6EC0BF0D8EC34F02981030193514A
:103480002D0AD8B446EF1AF00101299194C32FF107
:1034900095C330F196C331F197C332F198C333F13C
:1034A000E5EC34F05CEC34F000C10BF0A6EC0BF072
:1034B00001C10BF0A6EC0BF0D8EC34F0298103012C
:1034C0009A512D0AD8B467EF1AF0010129919BC3D4
:1034D0002FF19CC330F19DC331F19EC332F19FC3E4
:1034E00033F1E5EC34F05CEC34F000C10BF0A6EC09
:1034F0000BF001C10BF0A6EC0BF0D8EC34F02981F5
:103500000301A1512D0AD8B488EF1AF001012991C5
:10351000A2C32FF1A3C330F1A4C331F1A5C332F18B
:10352000A6C333F1E5EC34F05CEC34F000C10BF0F1
:10353000A6EC0BF001C10BF0A6EC0BF0D8EC34F0CC
:1035400029810301A8512D0AD8B4A9EF1AF001016D
:103550002991A9C32FF1AAC330F1ABC331F1ACC398
:1035600032F1ADC333F1E5EC34F05CEC34F000C182
:103570000BF0A6EC0BF001C10BF0A6EC0BF03E0E2D
:103580000C6EC4EC0BF0C4EC0BF0C4EC0BF0C4EC10
:103590000BF0C4EC0BF0C4EC0BF097EF23F003013D
:1035A0008351300AD8B43AEF1EF003018351310A37
:1035B000D8B467EF1FF003018351320AD8B4D5EFB6
:1035C0001FF003018351330AD8B4E5EF1FF0030164
:1035D0008351340AD8B4F5EF1FF003018351350A43
:1035E000D8B43BEF23F003018351360AD8B469EF16
:1035F00023F003018351370AD8B49CEF1DF0030177
:103600008351460AD8B48FEF22F0030183514D0A4B
:10361000D8B415EF1CF0030183516D0AD8B42FEF15
:103620001CF0030183515A0AD8B4E1EF1EF00301E4
:103630008351490AD8B469EF24F003018351500A39
:10364000D8B49BEF23F003018351540AD8B414EF8C
:1036500024F003018351630AD8B44FEF1CF0030137
:103660008351430AD8B447EF1DF003018351730A15
:10367000D8B44DEF1CF003018351610AD8B462EF56
:103680001BF003018351650AD8B48AEF1EF00301D1
:103690008351450AD8B498EF1EF003018351620AA2
:1036A000D8B4A6EF1EF003018351420AD8B4B4EF98
:1036B0001EF003018351760AD8B4C2EF1EF0D8A4DD
:1036C000ECEF2CF004014C0E826F35EC0FF004018E
:1036D000610E826F35EC0FF0E6EC36F004012C0E33
:1036E000826F35EC0FF097EC34F0ABC500F10101BF
:1036F0003AEC34F031C182F40401300E822735EC0B
:103700000FF032C182F40401300E822735EC0FF045
:1037100033C182F40401300E822735EC0FF004012E
:103720002C0E826F35EC0FF097EC34F0ACC500F145
:1037300001013AEC34F031C182F40401300E8227E9
:1037400035EC0FF032C182F40401300E822735ECE3
:103750000FF033C182F40401300E822735EC0FF0F4
:1037600004012C0E826F35EC0FF097EC34F0ADC5F0
:1037700000F101013AEC34F031C182F40401300E61
:10378000822735EC0FF032C182F40401300E82271B
:1037900035EC0FF033C182F40401300E822735EC92
:1037A0000FF004012C0E826F35EC0FF097EC34F023
:1037B000AEC500F101013AEC34F031C182F40401EC
:1037C000300E822735EC0FF032C182F40401300E46
:1037D000822735EC0FF033C182F40401300E8227CA
:1037E00035EC0FF004012C0E826F35EC0FF097ECE6
:1037F00034F0B2C500F101013AEC34F031C182F489
:103800000401300E822735EC0FF032C182F404013E
:10381000300E822735EC0FF033C182F40401300EF4
:10382000822735EC0FF097EF23F0D8EC34F084C307
:1038300033F1E5EC34F05CEC34F0200E0C6E00C19A
:103840000BF0A6EC0BF000C12FF505012F51000A7B
:1038500006E005012F51010A02E080EC37F0040177
:103860004C0E826F35EC0FF004014D0E826F35EC7B
:103870000FF004012C0E826F35EC0FF097EC34F052
:103880002FC500F13AEC34F033C182F40401300E5C
:10389000822735EC0FF097EF23F054EF3EF0040150
:1038A0004C0E826F35EC0FF00401630E826F35EC25
:1038B0000FF03EEC36F004012C0E826F35EC0FF069
:1038C00064EC1CF097EF23F097EC34F0B1C500F1F5
:1038D0000101003B0F0E00173AEC34F033C182F4C3
:1038E0000401300E822735EC0FF0B1C500F1010163
:1038F0000F0E010100173AEC34F033C182F40401D9
:10390000300E822735EC0FF004012D0E826F35EC5E
:103910000FF0B0C500F10101003B0F0E00173AECAB
:1039200034F033C182F40401300E822735EC0FF0FD
:10393000B0C500F101010F0E010100173AEC34F09F
:1039400033C182F40401300E822735EC0FF00401FC
:103950002D0E826F35EC0FF0AFC500F10101003B79
:103960000F0E00173AEC34F033C182F40401300E2C
:10397000822735EC0FF0AFC500F101010F0E0101F8
:1039800000173AEC34F033C182F40401300E822780
:1039900035EC0FF00401200E826F35EC0FF0AEC550
:1039A00000F10F0E010100173AEC34F033C182F43C
:1039B0000401300E822735EC0FF00401200E826FD7
:1039C00035EC0FF0ADC500F101010101003B0F0E18
:1039D00000173AEC34F033C182F40401300E822730
:1039E00035EC0FF0ADC500F101010F0E010100171C
:1039F0003AEC34F033C182F40401300E822735EC06
:103A00000FF004013A0E826F35EC0FF0ACC500F1F7
:103A10000101003B0F0E00173AEC34F033C182F481
:103A20000401300E822735EC0FF0ACC500F1010126
:103A30000F0E010100173AEC34F033C182F4040197
:103A4000300E822735EC0FF004013A0E826F35EC10
:103A50000FF0ABC500F10101003B0F0E00173AEC6F
:103A600034F033C182F40401300E822735EC0FF0BC
:103A7000ABC500F101010F0E00173AEC34F033C171
:103A800082F40401300E822735EC0FF0120084C35B
:103A9000E8FF0F0BE83AE8CFB1F585C3E8FF0F0B5D
:103AA0000501B11387C3E8FF0F0BE83AE8CFB0F583
:103AB00088C3E8FF0F0B0501B0138AC3E8FF0F0BA3
:103AC000E83AE8CFAFF58BC3E8FF0F0B0501AF1362
:103AD0008DC3E8FF0F0BE8CFAEF58FC3E8FF0F0BE8
:103AE000E83AE8CFADF590C3E8FF0F0B0501AD1341
:103AF00092C3E8FF0F0BE83AE8CFACF593C3E8FFB9
:103B00000F0B0501AC1395C3E8FF0F0BE83AE8CFA4
:103B1000ABF596C3E8FF0F0B0501AB1399EC36F03C
:103B200004014C0E826F35EC0FF00401430E826FDE
:103B300035EC0FF059EF1CF0078404014C0E826F36
:103B400035EC0FF00401370E826F35EC0FF00401F5
:103B50002C0E826F35EC0FF005012E51130A06E092
:103B600005012E51170A0DE037EF1EF00101000E7E
:103B7000006F000E016F100E026F000E036FCAEF90
:103B80001DF00101000E006F000E016F000E026FAC
:103B9000010E036F3AEC34F02AC182F40401300EB6
:103BA000822735EC0FF02BC182F40401300E8227FE
:103BB00035EC0FF02CC182F40401300E822735EC75
:103BC0000FF02DC182F40401300E822735EC0FF086
:103BD0002EC182F40401300E822735EC0FF02FC184
:103BE00082F40401300E822735EC0FF030C182F4EC
:103BF0000401300E822735EC0FF031C182F404014C
:103C0000300E822735EC0FF032C182F40401300E01
:103C1000822735EC0FF033C182F40401300E822785
:103C200035EC0FF004012C0E826F35EC0FF0010122
:103C3000200E006F000E016F000E026F000E036F6A
:103C40003AEC34F031C182F40401300E822735ECB5
:103C50000FF032C182F40401300E822735EC0FF0F0
:103C600033C182F40401300E822735EC0FF0079443
:103C700097EF23F0078415EC3EF097EC34F02DC558
:103C800000F13AEC34F004014C0E826F35EC0FF089
:103C90000401300E826F35EC0FF004012C0E826FA0
:103CA00035EC0FF031C182F40401300E822735EC7F
:103CB0000FF032C182F40401300E822735EC0FF090
:103CC00033C182F40401300E822735EC0FF0040179
:103CD0002C0E826F35EC0FF097EC34F02EC500F10E
:103CE0003AEC34F031C182F40401300E822735EC15
:103CF0000FF032C182F40401300E822735EC0FF050
:103D000033C182F40401300E822735EC0FF00794A2
:103D100097EF23F004014C0E826F35EC0FF0040195
:103D2000650E826F35EC0FF040EC38F097EF23F022
:103D300004014C0E826F35EC0FF00401450E826FCA
:103D400035EC0FF057EC38F097EF23F004014C0EF0
:103D5000826F35EC0FF00401620E826F35EC0FF0CC
:103D600085EC38F097EF23F004014C0E826F35ECB0
:103D70000FF00401420E826F35EC0FF06EEC38F05C
:103D800097EF23F004014C0E826F35EC0FF0040125
:103D9000760E826F35EC0FF004012C0E826F35EC3D
:103DA0000FF010A807D00401310E826F35EC0FF030
:103DB00097EF23F00401300E826F35EC0FF097EF90
:103DC00023F004014C0E826F35EC0FF004015A0E03
:103DD000826F35EC0FF004012C0E826F35EC0FF082
:103DE00015EC3EF097EC34F005012E51130A06E075
:103DF00005012E51170A0DE012EF1FF00101000E10
:103E0000006F000E016F100E026F000E036F12EFB5
:103E10001FF00101000E006F000E016F000E026F17
:103E2000010E036F0101200E046F000E056F000EDE
:103E3000066F000E076FCDEC33F03AEC34F02AC178
:103E400082F40401300E822735EC0FF02BC182F48E
:103E50000401300E822735EC0FF02CC182F40401EE
:103E6000300E822735EC0FF02DC182F40401300EA4
:103E7000822735EC0FF02EC182F40401300E822728
:103E800035EC0FF02FC182F40401300E822735EC9F
:103E90000FF030C182F40401300E822735EC0FF0B0
:103EA00031C182F40401300E822735EC0FF032C1AB
:103EB00082F40401300E822735EC0FF033C182F416
:103EC0000401300E822735EC0FF097EF23F00784C2
:103ED00004014C0E826F35EC0FF00401310E826F3D
:103EE00035EC0FF004012C0E826F35EC0FF025C578
:103EF00000F126C501F127C502F128C503F1010132
:103F0000200E046F000E056F000E066F000E076F87
:103F1000CDEC33F03AEC34F02AC182F40401300ED7
:103F2000822735EC0FF02BC182F40401300E82277A
:103F300035EC0FF02CC182F40401300E822735ECF1
:103F40000FF02DC182F40401300E822735EC0FF002
:103F50002EC182F40401300E822735EC0FF02FC100
:103F600082F40401300E822735EC0FF030C182F468
:103F70000401300E822735EC0FF031C182F40401C8
:103F8000300E822735EC0FF032C182F40401300E7E
:103F9000822735EC0FF033C182F40401300E822702
:103FA00035EC0FF0079497EF23F0078404014C0ED3
:103FB000826F35EC0FF00401320E826F35EC0FF09A
:103FC00073EC3AF0079497EF23F0078404014C0E4A
:103FD000826F35EC0FF00401330E826F35EC0FF079
:103FE000D0EC3AF0079472EF1FF0078404014C0EF6
:103FF000826F35EC0FF00401340E826F35EC0FF058
:1040000004012C0E826F35EC0FF0D8EC34F084C331
:104010002AF185C32BF186C32CF187C32DF188C308
:104020002EF189C32FF18AC330F18BC331F18CC3D8
:1040300032F18DC333F10101296BE5EC34F05CEC16
:1040400034F0200E046F000E056F000E066F000E98
:10405000076FADEC33F000C121F501C122F502C1BB
:1040600023F503C124F5C8EC3DF034C5ABF535C5E7
:10407000ACF536C5ADF537C5AEF538C5AFF539C5C4
:10408000B0F53AC5B1F564EC1CF004012C0E826F5A
:1040900035EC0FF03BC500F13CC501F13DC502F127
:1040A0003EC503F10101000E046F000E056F010E05
:1040B000066F000E076FCDEC33F03AEC34F0296751
:1040C00064EF20F069EF20F004012D0E826F35ECD3
:1040D0000FF030C182F40401300E822735EC0FF06E
:1040E00031C182F40401300E822735EC0FF0040157
:1040F0002E0E826F35EC0FF032C182F40401300EC7
:10410000822735EC0FF033C182F40401300E822790
:1041100035EC0FF004012C0E826F35EC0FF097ECAC
:1041200034F03FC500F140C501F116EC2EF004015A
:104130002C0E826F35EC0FF097EC34F041C500F196
:104140003AEC34F031C182F40401300E822735ECB0
:104150000FF032C182F40401300E822735EC0FF0EB
:1041600033C182F40401300E822735EC0FF00401D4
:104170002C0E826F35EC0FF00101036B026B48C50A
:1041800001F147C500F101AFCBEF20F00101FF0EB7
:10419000026FFF0E036F3AEC34F02967D2EF20F084
:1041A000D7EF20F004012D0E826F35EC0FF02FC1F8
:1041B00082F40401300E822735EC0FF030C182F416
:1041C0000401300E822735EC0FF031C182F4040176
:1041D000300E822735EC0FF032C182F40401300E2C
:1041E000822735EC0FF033C182F40401300E8227B0
:1041F00035EC0FF004012C0E826F35EC0FF001014D
:10420000036B026B4AC501F149C500F101AF0EEF26
:1042100021F00101FF0E026FFF0E036F3AEC34F044
:10422000296715EF21F01AEF21F004012D0E826F9E
:1042300035EC0FF02FC182F40401300E822735ECEB
:104240000FF030C182F40401300E822735EC0FF0FC
:1042500031C182F40401300E822735EC0FF032C1F7
:1042600082F40401300E822735EC0FF033C182F462
:104270000401300E822735EC0FF004012C0E826F02
:1042800035EC0FF00101036B026B4CC501F14BC51E
:1042900000F101AF51EF21F00101FF0E026FFF0E9F
:1042A000036F3AEC34F0296758EF21F05DEF21F00D
:1042B00004012D0E826F35EC0FF02FC182F4040142
:1042C000300E822735EC0FF030C182F40401300E3D
:1042D000822735EC0FF031C182F40401300E8227C1
:1042E00035EC0FF032C182F40401300E822735EC38
:1042F0000FF033C182F40401300E822735EC0FF049
:1043000004012C0E826F35EC0FF00101036B026B80
:104310004EC501F14DC500F101AF94EF21F001014F
:10432000FF0E026FFF0E036F3AEC34F029679BEF2C
:1043300021F0A0EF21F004012D0E826F35EC0FF07B
:104340002FC182F40401300E822735EC0FF030C10A
:1043500082F40401300E822735EC0FF031C182F473
:104360000401300E822735EC0FF032C182F40401D3
:10437000300E822735EC0FF033C182F40401300E89
:10438000822735EC0FF004012C0E826F35EC0FF014
:104390000101036B026B50C501F14FC500F101AF84
:1043A000D7EF21F00101FF0E026FFF0E036F3AEC11
:1043B00034F02967DEEF21F0E3EF21F004012D0E48
:1043C000826F35EC0FF02FC182F40401300E82278A
:1043D00035EC0FF030C182F40401300E822735EC49
:1043E0000FF031C182F40401300E822735EC0FF05A
:1043F00032C182F40401300E822735EC0FF033C154
:1044000082F40401300E822735EC0FF004012C0EEB
:10441000826F35EC0FF00101036B026B52C501F1A5
:1044200051C500F101AF1AEF22F00101FF0E026F3A
:10443000FF0E036F3AEC34F0296721EF22F026EFEC
:1044400022F004012D0E826F35EC0FF02FC182F4A3
:104450000401300E822735EC0FF030C182F40401E4
:10446000300E822735EC0FF031C182F40401300E9A
:10447000822735EC0FF032C182F40401300E82271E
:1044800035EC0FF033C182F40401300E822735EC95
:104490000FF004012C0E826F35EC0FF00101036B5D
:1044A000026B46C501F145C500F101AF5DEF22F099
:1044B0000101FF0E026FFF0E036F3AEC34F0296723
:1044C00064EF22F069EF22F004012D0E826F35ECCB
:1044D0000FF02FC182F40401300E822735EC0FF06B
:1044E00030C182F40401300E822735EC0FF031C167
:1044F00082F40401300E822735EC0FF032C182F4D1
:104500000401300E822735EC0FF033C182F4040130
:10451000300E822735EC0FF0079497EF23F0D8EC9C
:1045200034F085C32AF186C32BF187C32CF188C3ED
:104530002DF189C32EF18AC32FF18BC330F18CC3C7
:1045400031F18DC332F18EC333F10101296BE5ECFA
:1045500034F05CEC34F00101010E046F000E056FC5
:10456000000E066F000E076F9CEC33F0100E046F08
:10457000000E056F000E066F000E076FADEC33F0F6
:1045800000C129F501C12AF502C12BF503C12CF5A3
:10459000FAEC39F004014C0E826F35EC0FF0040197
:1045A000460E826F35EC0FF004012C0E826F35EC55
:1045B0000FF025C500F126C501F127C502F128C578
:1045C00003F10101100E046F000E056F000E066F5F
:1045D000000E076FCDEC33F03AEC34F02AC182F4D0
:1045E0000401300E822735EC0FF02BC182F4040158
:1045F000300E822735EC0FF02CC182F40401300E0E
:10460000822735EC0FF02DC182F40401300E822791
:1046100035EC0FF02EC182F40401300E822735EC08
:104620000FF02FC182F40401300E822735EC0FF019
:1046300030C182F40401300E822735EC0FF031C115
:1046400082F40401300E822735EC0FF032C182F47F
:104650000401300E822735EC0FF033C182F40401DF
:10466000300E822735EC0FF097EF23F00F98D0EC47
:104670003AF0ECEF2CF004014C0E826F35EC0FF0A9
:104680000401350E826F35EC0FF004012C0E826FA1
:1046900035EC0FF097EC34F00784B5C500F10794C2
:1046A0003AEC34F031C182F40401300E822735EC4B
:1046B0000FF032C182F40401300E822735EC0FF086
:1046C00033C182F40401300E822735EC0FF097EFEE
:1046D00023F093EC3AF097EC34F033C500F13AEC68
:1046E00034F004014C0E826F35EC0FF00401360EED
:1046F000826F35EC0FF004012C0E826F35EC0FF059
:1047000031C182F40401300E822735EC0FF032C142
:1047100082F40401300E822735EC0FF033C182F4AD
:104720000401300E822735EC0FF097EF23F03FECB9
:104730000FF0ECEF2CF004014C0E826F35EC0FF013
:104740000401500E826F35EC0FF004012C0E826FC5
:1047500035EC0FF085C32AF186C32BF187C32CF10A
:1047600088C32DF189C32EF18AC32FF18BC330F199
:104770008CC331F18DC332F18EC333F10101E5EC0D
:1047800034F05CEC34F003018451530A0DE0030172
:1047900084514D0A38E00401780E826F35EC0FF039
:1047A0003FEC0FF0ECEF2CF00401530E826F35EC70
:1047B0000FF0250E0C6E00C10BF0A6EC0BF0260ED0
:1047C0000C6E01C10BF0A6EC0BF0270E0C6E02C1B3
:1047D0000BF0A6EC0BF0280E0C6E03C10BF0A6EC50
:1047E0000BF000C153F501C154F502C155F503C1E9
:1047F00056F500C157F501C158F502C159F503C17D
:104800005AF578EF24F004014D0E826F35EC0FF06D
:10481000290E0C6E00C10BF0A6EC0BF000C15BF58D
:1048200000C15CF578EF24F004014C0E826F35EC8A
:104830000FF00401540E826F35EC0FF004012C0EC2
:10484000826F35EC0FF084C32AF185C32BF186C348
:104850002CF187C32DF188C32EF189C32FF18AC3B0
:1048600030F18BC331F18DC332F18EC333F10101CD
:10487000E5EC34F05CEC34F00101000E046F000E46
:10488000056F010E066F000E076FADEC33F0210EC1
:104890000C6E00C10BF0A6EC0BF0220E0C6E01C1E9
:1048A0000BF0A6EC0BF0230E0C6E02C10BF0A6EC85
:1048B0000BF0240E0C6E03C10BF0A6EC0BF000C144
:1048C0005DF501C15EF502C15FF503C160F578EFEA
:1048D00024F004014C0E826F35EC0FF00401490EF8
:1048E000826F35EC0FF004012C0E826F35EC0FF067
:1048F000250EBDEC0BF0E8CF00F1260EBDEC0BF061
:10490000E8CF01F1270EBDEC0BF0E8CF02F1280E45
:10491000BDEC0BF0E8CF03F13AEC34F01DEC32F0D3
:104920000401730E826F35EC0FF004012C0E826FC0
:1049300035EC0FF097EC34F0290EBDEC0BF0E8CF1E
:1049400000F13AEC34F01DEC32F00401730E826F8A
:1049500035EC0FF004012C0E826F35EC0FF057C5CB
:1049600000F158C501F159C502F15AC503F13AECFD
:1049700034F01DEC32F00401730E826F35EC0FF051
:1049800004012C0E826F35EC0FF097EC34F05CC50F
:1049900000F13AEC34F01DEC32F004016D0E826F40
:1049A00035EC0FF004012C0E826F35EC0FF05DC575
:1049B00000F15EC501F15FC502F160C503F107ECCE
:1049C0002DF004012C0E826F35EC0FF03FEC0FF050
:1049D000ECEF2CF083C32AF184C32BF185C32CF1B7
:1049E00086C32DF187C32EF188C32FF189C330F11F
:1049F0008AC331F18BC332F18CC333F10101E5EC91
:104A000034F05CEC34F0160E0C6E00C10BF0A6EC2A
:104A10000BF0170E0C6E01C10BF0A6EC0BF0180E8C
:104A20000C6E02C10BF0A6EC0BF0190E0C6E03C15C
:104A30000BF0A6EC0BF000C18AF101C18BF102C1B1
:104A40008CF103C18DF100C18EF101C18FF102C162
:104A500090F103C191F1CCEF25F083C32AF184C317
:104A60002BF185C32CF186C32DF187C32EF188C3AA
:104A70002FF189C330F18AC331F18BC332F18CC37A
:104A800033F10101E5EC34F05CEC34F000C18AF163
:104A900001C18BF102C18CF103C18DF100C18EF116
:104AA00001C18FF102C190F103C191F1CCEF25F06A
:104AB00083C32AF184C32BF185C32CF186C32DF166
:104AC00087C32EF188C32FF189C330F18AC331F136
:104AD0008CC332F18DC333F10101E5EC34F05CECB1
:104AE00034F00101000E046F000E056F010E066F19
:104AF000000E076FADEC33F01A0E0C6E00C10BF018
:104B0000A6EC0BF01B0E0C6E01C10BF0A6EC0BF02B
:104B10001C0E0C6E02C10BF0A6EC0BF01D0E0C6E01
:104B200003C10BF0A6EC0BF000C192F101C193F1AF
:104B300002C194F103C195F1CCEF25F083C32AF1B2
:104B400084C32BF185C32CF186C32DF187C32EF1CD
:104B500088C32FF189C330F18AC331F18CC332F19C
:104B60008DC333F10101E5EC34F05CEC34F001016C
:104B7000000E046F000E056F010E066F000E076F2A
:104B8000ADEC33F000C192F101C193F102C194F197
:104B900003C195F1CCEF25F0160EBDEC0BF0E8CF7C
:104BA00000F1170EBDEC0BF0E8CF01F1180EBDECD3
:104BB0000BF0E8CF02F1190EBDEC0BF0E8CF03F1DA
:104BC0003AEC34F01DEC32F00401730E826F35ECD8
:104BD0000FF004012C0E826F35EC0FF08AC100F14A
:104BE0008BC101F18CC102F18DC103F13AEC34F0BB
:104BF0001DEC32F00401730E826F35EC0FF00401EE
:104C00002C0E826F35EC0FF01A0EBDEC0BF0E8CFD6
:104C100000F11B0EBDEC0BF0E8CF01F11C0EBDEC5A
:104C20000BF0E8CF02F11D0EBDEC0BF0E8CF03F165
:104C300007EC2DF004012C0E826F35EC0FF092C1C1
:104C400000F193C101F194C102F195C103F107ECA8
:104C50002DF03FEC0FF0ECEF2CF00401690E826FA9
:104C600035EC0FF004012C0E826F35EC0FF00101D2
:104C7000040E006F000E016F000E026F000E036F36
:104C80003AEC34F02CC182F40401300E822735EC6A
:104C90000FF02DC182F40401300E822735EC0FF0A5
:104CA0002EC182F40401300E822735EC0FF02FC1A3
:104CB00082F40401300E822735EC0FF030C182F40B
:104CC0000401300E822735EC0FF031C182F404016B
:104CD000300E822735EC0FF032C182F40401300E21
:104CE000822735EC0FF033C182F40401300E8227A5
:104CF00035EC0FF004012C0E826F35EC0FF0010142
:104D00000B0E006F000E016F000E026F000E036F9E
:104D10003AEC34F02CC182F40401300E822735ECD9
:104D20000FF02DC182F40401300E822735EC0FF014
:104D30002EC182F40401300E822735EC0FF02FC112
:104D400082F40401300E822735EC0FF030C182F47A
:104D50000401300E822735EC0FF031C182F40401DA
:104D6000300E822735EC0FF032C182F40401300E90
:104D7000822735EC0FF033C182F40401300E822714
:104D800035EC0FF004012C0E826F35EC0FF00101B1
:104D90002C0E006F000E016F000E026F000E036FED
:104DA0003AEC34F02CC182F40401300E822735EC49
:104DB0000FF02DC182F40401300E822735EC0FF084
:104DC0002EC182F40401300E822735EC0FF02FC182
:104DD00082F40401300E822735EC0FF030C182F4EA
:104DE0000401300E822735EC0FF031C182F404014A
:104DF000300E822735EC0FF032C182F40401300E00
:104E0000822735EC0FF033C182F40401300E822783
:104E100035EC0FF004012C0E826F35EC0FF0200EF4
:104E2000F86EF76AF66A04010900F5CF82F435ECF2
:104E30000FF00900F5CF82F435EC0FF00900F5CF43
:104E400082F435EC0FF00900F5CF82F435EC0FF069
:104E50000900F5CF82F435EC0FF00900F5CF82F4AC
:104E600035EC0FF00900F5CF82F435EC0FF00900B6
:104E7000F5CF82F435EC0FF03FEC0FF0ECEF2CF0B7
:104E80008351630AD8A4ECEF2CF08451610AD8A4B2
:104E9000ECEF2CF085516C0AD8A4ECEF2CF0865185
:104EA000410A3FE08651440A1BE08651420AD8B4C9
:104EB000A4EF27F08651350AD8B476EF2EF086514C
:104EC000360AD8B4CBEF2EF08651370AD8B434EF77
:104ED0002FF08651380AD8B492EF2FF0ECEF2CF077
:104EE0000798079A04017A0E826F35EC0FF00401DF
:104EF000780E826F35EC0FF00401640E826F35EC92
:104F00000FF00401550E826F35EC0FF08DEF27F096
:104F100004014C0E826F35EC0FF03FEC0FF0ECEF1C
:104F20002CF00788079A04017A0E826F35EC0FF097
:104F30000401410E826F35EC0FF00401610E826FA7
:104F400035EC0FF081EF27F00798078A04017A0EFD
:104F5000826F35EC0FF00401420E826F35EC0FF0DA
:104F60000401610E826F35EC0FF081EF27F0010133
:104F70006667C2EF27F06767C2EF27F06867C2EF86
:104F800027F0696715D04F67CDEF27F05067CDEF59
:104F900027F05167CDEF27F052670AD00101000ECC
:104FA000006F000E016F000E026F000E036F120003
:104FB00011B80AD00101620E046F010E056F000ED8
:104FC000066F000E076F09D00101A70E046F020ED5
:104FD000056F000E066F000E076F66C100F167C116
:104FE00001F168C102F169C103F19CEC33F003BF28
:104FF0006AEF28F0119A119C0101000E046FA80EAF
:10500000056F550E066F020E076F66C100F167C18E
:1050100001F168C102F169C103F166C186F167C19E
:1050200087F168C188F169C189F19CEC33F003BF55
:105030000BD00101000E866FA80E876F550E886F8A
:10504000020E896F118A119C0E0EBDEC0BF0E8CF99
:1050500018F10F0EBDEC0BF0E8CF19F1100EBDECFE
:105060000BF0E8CF1AF1110EBDEC0BF0E8CF1BF1FD
:10507000E5EC32F086C104F187C105F188C106F183
:1050800089C107F19CEC33F00782A9EC32F0E5EC22
:1050900032F00792A9EC32F086C100F187C101F12C
:1050A00088C102F189C103F10792A9EC32F0CC0E5C
:1050B000046FE00E056F870E066F050E076F9CEC00
:1050C00033F000C118F101C119F102C11AF103C195
:1050D0001BF13BD0119C119A0101800E006F1A0E3A
:1050E000016F060E026F000E036F4FC104F150C135
:1050F00005F151C106F152C107F19CEC33F003AF49
:1051000005D097EC34F0118C119A12000E0EBDEC04
:105110000BF0E8CF18F10F0EBDEC0BF0E8CF19F152
:10512000100EBDEC0BF0E8CF1AF1110EBDEC0BF038
:10513000E8CF1BF14FC100F150C101F151C102F1A3
:1051400052C103F10782A9EC32F018C100F119C174
:1051500001F11AC102F11BC103F112000401730E27
:10516000826F35EC0FF004012C0E826F35EC0FF0DE
:10517000078462C166F163C167F164C168F165C10A
:1051800069F14BC14FF14CC150F14DC151F14EC1CC
:1051900052F157C159F158C15AF10794D4EC28F093
:1051A0003FEC0FF0ECEF2CF066C100F167C101F1AC
:1051B00068C102F169C103F101013AEC34F01DEC60
:1051C00032F00401630E826F35EC0FF004012C0EF7
:1051D000826F35EC0FF04FC100F150C101F151C1A8
:1051E00002F152C103F101013AEC34F01DEC32F04E
:1051F0000401660E826F35EC0FF004012C0E826FF5
:1052000035EC0FF097EC34F059C100F15AC101F1BF
:1052100001013AEC34F01DEC32F00401740E826F9F
:1052200035EC0FF0120010820401530E826F35EC42
:105230000FF004012C0E826F35EC0FF083C32AF1BE
:1052400084C32BF185C32CF186C32DF187C32EF1C6
:1052500088C32FF189C330F18AC331F18BC332F196
:105260008CC333F10101E5EC34F05CEC34F000C1A7
:1052700066F101C167F102C168F103C169F18EC332
:105280002AF18FC32BF190C32CF191C32DF192C35E
:105290002EF193C32FF194C330F195C331F196C32E
:1052A00032F197C333F10101E5EC34F05CEC34F0FA
:1052B00000C14FF101C150F102C151F103C152F1DE
:1052C000D8EC34F099C32FF19AC330F19BC331F17C
:1052D0009CC332F19DC333F10101E5EC34F05CEC89
:1052E00034F000C159F101C15AF1D4EC28F00401A5
:1052F0002C0E826F35EC0FF08BEF29F0118E18B069
:10530000108C17BE02D017A4108E8251520A02E1EF
:105310000F8201D00F928251750A02E1108401D0F0
:1053200010948251550A02E1108601D0109611A006
:1053300003D011A401D01084078410B2F9EF29F032
:1053400010A4E5EF29F0B6C166F1B7C167F1B8C1A5
:1053500068F1B9C169F1BAC16AF1BBC16BF1BCC1F5
:105360006CF1BDC16DF1BEC16EF1BFC16FF1C0C1C5
:1053700070F1C1C171F1C2C172F1C3C173F1C4C195
:1053800074F1C5C175F1C6C176F1C7C177F1C8C165
:1053900078F1C9C179F1CAC17AF1CBC17BF1CCC135
:1053A0007CF1CDC17DF1CEC17EF1CFC17FF1D0C105
:1053B00080F1D1C181F1D2C182F1D3C183F1D4C1D5
:1053C00084F1D5C185F1EDEF29F062C166F163C1C9
:1053D00067F164C168F165C169F14BC14FF14CC11E
:1053E00050F14DC151F14EC152F157C159F158C15F
:1053F0005AF107940FA01BEF2AF00101926708EF02
:105400002AF0936708EF2AF0946708EF2AF095676F
:105410000CEF2AF01BEF2AF0B7EC27F092C104F151
:1054200093C105F194C106F195C107F19CEC33F0ED
:1054300003BFB2EF2CF0B7EC27F00101000E046FB0
:10544000000E056F010E066F000E076FCDEC33F0F6
:1054500011A02CD011A22AD03AEC34F0296701D047
:1054600007D004012D0E826F35EC0FF0B0EF2CF059
:1054700030C182F40401300E822735EC0FF031C1C7
:1054800082F40401300E822735EC0FF032C182F431
:105490000401300E822735EC0FF033C182F4040191
:1054A000300E822735EC0FF0B0EF2CF012A8C5D0EB
:1054B000129819C01AF01A3A1A42070E1A16000169
:1054C0001A50000AD8B4E9EF2AF000011A50010A74
:1054D000D8B475EF2AF000011A50020AD8B473EF5D
:1054E0002AF01BEF2BF01BEF2BF097EC34F029C0C8
:1054F00001F12AC000F1D89001330033D890013374
:1055000000330101630E046F000E056F000E066F7D
:10551000000E076FCDEC33F0280E046F000E056F00
:10552000000E066F000E076F9CEC33F000C12CF0EC
:1055300097EC34F027C001F1019F019D28C000F1D4
:105540000101A40E046F000E056F000E066F000E21
:10555000076FCDEC33F000C12BF000C104F101C1A5
:1055600005F102C106F103C107F1640E006F000EE0
:10557000016F000E026F000E036F9CEC33F0050EFE
:10558000046F000E056F000E066F000E076FCDEC66
:1055900033F000C104F101C105F102C106F103C1FC
:1055A00007F197EC34F02CC000F19CEC33F000C113
:1055B0002DF02DC0E8FF050F2C5C03E78A841BEF5C
:1055C0002BF02DC0E8FF0A0F2C5C01E68A941BEF3C
:1055D0002BF000C124F101C125F102C126F103C164
:1055E00027F197EC34F09DEC34F019501F0BE8CF05
:1055F00000F10101640E046F000E056F000E066FCE
:10560000000E076FADEC33F024C104F125C105F1A4
:1056100026C106F127C107F19CEC33F003BF02D08D
:105620008A9401D08A8424C100F125C101F126C1E8
:1056300002F127C103F1B2EF2CF000C124F101C146
:1056400025F102C126F103C127F110AE4CD0109E06
:1056500000C108F101C109F102C10AF103C10BF156
:105660003AEC34F030C1D6F131C1D7F132C1D8F1C2
:1056700033C1D9F108C100F109C101F10AC102F138
:105680000BC103F101016C0E046F070E056F000ED4
:10569000066F000E076F9CEC33F003BF04D00101CE
:1056A000550EDA6F1CD008C100F109C101F10AC121
:1056B00002F10BC103F10101A40E046F060E056F88
:1056C000000E066F000E076F9CEC33F003BF04D092
:1056D00001017F0EDA6F03D00101FF0EDA6F1B8E1E
:1056E00011AEB2EF2CF024C100F125C101F126C1A9
:1056F00002F127C103F110A485EF2BF00401750E10
:10570000826F35EC0FF08AEF2BF00401720E826F7E
:1057100035EC0FF004012C0E826F35EC0FF03AECF3
:1057200034F0296799EF2BF00401200E826F9CEF73
:105730002BF004012D0E826F35EC0FF030C182F496
:105740000401300E822735EC0FF031C182F40401E0
:10575000300E822735EC0FF004012E0E826F35ECEF
:105760000FF032C182F40401300E822735EC0FF0C5
:1057700033C182F40401300E822735EC0FF00401AE
:105780006D0E826F35EC0FF004012C0E826F35EC3C
:105790000FF04FC100F150C101F151C102F152C1EE
:1057A00003F101013AEC34F01DEC32F00401480E33
:1057B000826F35EC0FF004017A0E826F35EC0FF03A
:1057C00004012C0E826F35EC0FF066C100F167C149
:1057D00001F168C102F169C103F101013AEC34F051
:1057E0001DEC32F00401630E826F35EC0FF0040102
:1057F0002C0E826F35EC0FF066C100F167C101F12C
:1058000068C102F169C103F101010A0E046F000EC3
:10581000056F000E066F000E076FADEC33F0000E43
:10582000046F120E056F000E066F000E076FCDECB1
:1058300033F03AEC34F02AC182F40401300E8227AE
:1058400035EC0FF02BC182F40401300E822735ECC9
:105850000FF02CC182F40401300E822735EC0FF0DA
:105860002DC182F40401300E822735EC0FF02EC1D9
:1058700082F40401300E822735EC0FF02FC182F440
:105880000401300E822735EC0FF030C182F40401A0
:10589000300E822735EC0FF004012E0E826F35ECAE
:1058A0000FF031C182F40401300E822735EC0FF085
:1058B00032C182F40401300E822735EC0FF033C17F
:1058C00082F40401300E822735EC0FF00401730ED0
:1058D000826F35EC0FF004012C0E826F35EC0FF067
:1058E00097EC34F059C100F15AC101F116EC2EF0D9
:1058F0000FB27EEF2CF00FA0B0EF2CF004012C0EB5
:10590000826F35EC0FF0200EF86EF76AF66A04012C
:105910000900F5CF82F435EC0FF00900F5CF82F4E1
:1059200035EC0FF00900F5CF82F435EC0FF00900EB
:10593000F5CF82F435EC0FF00900F5CF82F435ECA9
:105940000FF00900F5CF82F435EC0FF00900F5CF28
:1059500082F435EC0FF00900F5CF82F435EC0FF04E
:105960003FEC0FF00F90ECEF2CF00401630E826F10
:1059700035EC0FF004012C0E826F35EC0FF0F2ECD9
:105980002CF004012C0E826F35EC0FF065EC2DF03D
:1059900004012C0E826F35EC0FF0E1EC2DF00401C8
:1059A0002C0E826F35EC0FF00101F80E006FCD0E5A
:1059B000016F660E026F030E036F07EC2DF00401FA
:1059C0002C0E826F35EC0FF0F7EC2DF03FEC0FF062
:1059D000ECEF2CF03FEC0FF00301C26B079010923C
:1059E000FBEF2FF0D8900E0EBDEC0BF0E8CF00F1DE
:1059F0000F0EBDEC0BF0E8CF01F1100EBDEC0BF07B
:105A0000E8CF02F1110EBDEC0BF0E8CF03F101017C
:105A1000000E046F000E056F010E066F000E076F7B
:105A2000CDEC33F03AEC34F02AC182F40401300EAC
:105A3000822735EC0FF02BC182F40401300E82274F
:105A400035EC0FF02CC182F40401300E822735ECC6
:105A50000FF02DC182F40401300E822735EC0FF0D7
:105A60002EC182F40401300E822735EC0FF02FC1D5
:105A700082F40401300E822735EC0FF030C182F43D
:105A80000401300E822735EC0FF031C182F404019D
:105A9000300E822735EC0FF004012E0E826F35ECAC
:105AA0000FF032C182F40401300E822735EC0FF082
:105AB00033C182F40401300E822735EC0FF004016B
:105AC0006D0E826F35EC0FF01200120EBDEC0BF074
:105AD000E8CF00F1130EBDEC0BF0E8CF01F1140E8E
:105AE000BDEC0BF0E8CF02F1150EBDEC0BF0E8CFEA
:105AF00003F101010A0E046F000E056F000E066F20
:105B0000000E076FADEC33F0000E046F120E056F40
:105B1000000E066F000E076FCDEC33F03AEC34F058
:105B20002AC182F40401300E822735EC0FF02BC11C
:105B300082F40401300E822735EC0FF02CC182F480
:105B40000401300E822735EC0FF02DC182F40401E0
:105B5000300E822735EC0FF02EC182F40401300E96
:105B6000822735EC0FF02FC182F40401300E82271A
:105B700035EC0FF030C182F40401300E822735EC91
:105B80000FF004012E0E826F35EC0FF031C182F45C
:105B90000401300E822735EC0FF032C182F404018B
:105BA000300E822735EC0FF033C182F40401300E41
:105BB000822735EC0FF00401730E826F35EC0FF085
:105BC00012000A0EBDEC0BF0E8CF00F10B0EBDEC9D
:105BD0000BF0E8CF01F10C0EBDEC0BF0E8CF02F1B9
:105BE0000D0EBDEC0BF0E8CF03F116EF2EF0060E14
:105BF000BDEC0BF0E8CF00F1070EBDEC0BF0E8CFE9
:105C000001F1080EBDEC0BF0E8CF02F1090EBDEC7E
:105C10000BF0E8CF03F116EF2EF0010197EC34F012
:105C2000078457C100F158C101F107940101E80E42
:105C3000046F800E056F000E066F000E076FADEC4F
:105C400033F0000E046F040E056F000E066F000E99
:105C5000076FCDEC33F0880E046F130E056F000E46
:105C6000066F000E076F9CEC33F00A0E046F000EF7
:105C7000056F000E066F000E076FCDEC33F03AECA7
:105C800034F0010129674AEF2EF00401200E826FE3
:105C90004DEF2EF004012D0E826F35EC0FF030C168
:105CA00082F40401300E822735EC0FF031C182F40A
:105CB0000401300E822735EC0FF032C182F404016A
:105CC000300E822735EC0FF004012E0E826F35EC7A
:105CD0000FF033C182F40401300E822735EC0FF04F
:105CE0000401430E826F35EC0FF0120087C32AF1D6
:105CF00088C32BF189C32CF18AC32DF18BC32EF1FC
:105D00008CC32FF18DC330F18EC331F190C332F1CA
:105D100091C333F10101296BE5EC34F05CEC34F014
:105D20000101000E046F000E056F010E066F000EDC
:105D3000076FADEC33F00E0E0C6E00C10BF0A6EC4D
:105D40000BF00F0E0C6E01C10BF0A6EC0BF0100E59
:105D50000C6E02C10BF0A6EC0BF0110E0C6E03C121
:105D60000BF0A6EC0BF004017A0E826F35EC0FF00D
:105D700004012C0E826F35EC0FF00401350E826F9A
:105D800035EC0FF004012C0E826F35EC0FF0F2ECC5
:105D90002CF08DEF27F087C32AF188C32BF189C33C
:105DA0002CF18AC32DF18BC32EF18CC32FF18DC33F
:105DB00030F18EC331F190C332F191C333F101015F
:105DC000296BE5EC34F05CEC34F0880E046F130EB4
:105DD000056F000E066F000E076FA1EC33F0000E8A
:105DE000046F040E056F000E066F000E076FADEC1A
:105DF00033F00101E80E046F800E056F000E066F90
:105E0000000E076FCDEC33F00A0E0C6E00C10BF0E4
:105E1000A6EC0BF00B0E0C6E01C10BF0A6EC0BF018
:105E20000C0E0C6E02C10BF0A6EC0BF00D0E0C6EFE
:105E300003C10BF0A6EC0BF004017A0E826F35EC77
:105E40000FF004012C0E826F35EC0FF00401360EBA
:105E5000826F35EC0FF004012C0E826F35EC0FF0E1
:105E6000E1EC2DF08DEF27F087C32AF188C32BF1E9
:105E700089C32CF18AC32DF18BC32EF18CC32FF172
:105E80008DC330F18FC331F190C332F191C333F13F
:105E90000101E5EC34F05CEC34F0000E046F120EFE
:105EA000056F000E066F000E076FADEC33F00101B9
:105EB0000A0E046F000E056F000E066F000E076FCE
:105EC000CDEC33F0120E0C6E00C10BF0A6EC0BF013
:105ED000130E0C6E01C10BF0A6EC0BF0140E0C6E41
:105EE00002C10BF0A6EC0BF0150E0C6E03C10BF00B
:105EF000A6EC0BF004017A0E826F35EC0FF0040172
:105F00002C0E826F35EC0FF00401370E826F35ECEA
:105F10000FF004012C0E826F35EC0FF065EC2DF0C4
:105F20008DEF27F087C32AF188C32BF189C32CF1A9
:105F30008AC32DF18BC32EF18CC32FF18DC330F1A9
:105F40008EC331F190C332F191C333F10101296B5A
:105F5000E5EC34F05CEC34F0880E046F130E056F42
:105F6000000E066F000E076FA1EC33F0000E046FF9
:105F7000040E056F000E066F000E076FADEC33F0D8
:105F80000101E80E046F800E056F000E066F000E13
:105F9000076FCDEC33F0060E0C6E00C10BF0A6ECD3
:105FA0000BF0070E0C6E01C10BF0A6EC0BF0080E07
:105FB0000C6E02C10BF0A6EC0BF0090E0C6E03C1C7
:105FC0000BF0A6EC0BF004017A0E826F35EC0FF0AB
:105FD00004012C0E826F35EC0FF00401380E826F35
:105FE00035EC0FF004012C0E826F35EC0FF0F7EC5E
:105FF0002DF08DEF27F007A86FEF30F00101800E34
:10600000006F1A0E016F060E026F000E036F4BC178
:1060100004F14CC105F14DC106F14EC107F19CECF4
:1060200033F003BFB6EF30F017EC32F04BC100F1A4
:106030004CC101F14DC102F14EC103F10782A9EC3F
:1060400032F018C104F119C105F11AC106F11BC1E2
:1060500007F1F80E006FCD0E016F660E026F030E92
:10606000036F9CEC33F00E0E0C6E00C10BF0A6EC2F
:106070000BF00F0E0C6E01C10BF0A6EC0BF0100E26
:106080000C6E02C10BF0A6EC0BF0110E0C6E03C1EE
:106090000BF0A6EC0BF00784010197EC34F057C12C
:1060A00000F158C101F107940A0E0C6E00C10BF00B
:1060B000A6EC0BF00B0E0C6E01C10BF0A6EC0BF076
:1060C0000C0E0C6E02C10BF0A6EC0BF00D0E0C6E5C
:1060D00003C10BF0A6EC0BF00798B6EF30F007AA5F
:1060E000B6EF30F00784010197EC34F057C100F1AE
:1060F00058C101F10794060E0C6E00C10BF0A6EC1E
:106100000BF0070E0C6E01C10BF0A6EC0BF0080EA5
:106110000C6E02C10BF0A6EC0BF0090E0C6E03C165
:106120000BF0A6EC0BF0078462C100F163C101F132
:1061300064C102F165C103F10794120E0C6E00C137
:106140000BF0A6EC0BF0130E0C6E01C10BF0A6ECDD
:106150000BF0140E0C6E02C10BF0A6EC0BF0150E3A
:106160000C6E03C10BF0A6EC0BF0079A04018051F2
:1061700081197F0B0BE09EA809D014EE00F081512D
:106180007F0BE126E750812B0F01AD6E05012F51EA
:10619000010A13E081AADDEF30F005012F51000A5A
:1061A0000AE00FB8DDEF30F005013067DDEF30F0C9
:1061B0000FB8DDEF30F054EF3EF081B8F2EF30F081
:1061C000E6EC36F005012F51020A02E0F2EF30F062
:1061D0005C2FF2EF30F05BC55CF50501010E306F0E
:1061E0003C0E316F84EF0EF006013251385D3351B1
:1061F000D8A0010F395D800BD8A403EF31F032C66F
:1062000038F633C639F6120006013251365D335185
:10621000D8A0010F375D800BD8B413EF31F032C630
:1062200036F633C637F6120007841AC632F61BC696
:1062300033F61CC638F61DC639F6F4EC30F01EC62F
:1062400032F61FC633F6F4EC30F020C632F621C623
:1062500033F6F4EC30F01AC632F61BC633F61CC621
:1062600036F61DC637F604EC31F01EC632F61FC6F0
:1062700033F604EC31F020C632F621C633F604ECD6
:1062800031F03851365F3951D8A03929375F97EC52
:1062900034F036C600F137C601F1A3EC34F000C18A
:1062A0003AF601C13BF622C632F623C633F624C6BF
:1062B00038F625C639F6F4EC30F026C632F627C695
:1062C00033F6F4EC30F028C632F629C633F6F4EC97
:1062D00030F022C632F623C633F624C636F625C67B
:1062E00037F604EC31F026C632F627C633F604EC56
:1062F00031F028C632F629C633F604EC31F03851B5
:10630000365F3951D8A03929375F97EC34F036C65B
:1063100000F137C601F1A3EC34F000C13CF601C135
:106320003DF62AC632F62BC633F62CC638F62DC6F5
:1063300039F6F4EC30F02EC632F62FC633F6F4EC14
:1063400030F030C632F631C633F6F4EC30F02AC6FF
:1063500032F62BC633F62CC636F62DC637F604ECCD
:1063600031F02EC632F62FC633F604EC31F030C6CB
:1063700032F631C633F604EC31F03851365F39511C
:10638000D8A03929375F97EC34F036C600F137C60C
:1063900001F1A3EC34F000C13EF601C13FF63AC66C
:1063A00032F63BC633F63CC636F63DC637F604EC4D
:1063B00031F03EC632F63FC633F604EC31F00794B6
:1063C000120018C100F119C101F11AC102F11BC17B
:1063D00003F1000E046F000E056F010E066F000E34
:1063E000076FCDEC33F029A10CEF32F02051D8B477
:1063F0000CEF32F018C100F119C101F11AC102F11C
:106400001BC103F1000E046F000E056F0A0E066F2C
:10641000000E076FCDEC33F01200010104510013A0
:106420000551011306510213075103131200010114
:10643000186B196B1A6B1B6B12002AC182F40401D2
:10644000300E822735EC0FF02BC182F40401300EA0
:10645000822735EC0FF02CC182F40401300E822724
:1064600035EC0FF02DC182F40401300E822735EC9B
:106470000FF02EC182F40401300E822735EC0FF0AC
:106480002FC182F40401300E822735EC0FF030C1A9
:1064900082F40401300E822735EC0FF031C182F412
:1064A0000401300E822735EC0FF032C182F4040172
:1064B000300E822735EC0FF033C182F40401300E28
:1064C000822735EC0FF012002FC182F40401300E48
:1064D000822735EC0FF030C182F40401300E8227A0
:1064E00035EC0FF031C182F40401300E822735EC17
:1064F0000FF032C182F40401300E822735EC0FF028
:1065000033C182F40401300E822735EC0FF0120003
:10651000060E1D6E060E1E6E060E1F6E1D2E8EEFD3
:1065200032F01E2E8EEF32F01F2E8EEF32F08B8463
:10653000020E1D6E020E1E6E020E1F6E1D2E9EEFAF
:1065400032F01E2E9EEF32F01F2E9EEF32F08B9413
:1065500012000101005305E1015303E1025301E17F
:10656000002B6CEC33F097EC34F03951006F3A515A
:10657000016F420E046F4B0E056F000E066F000E8A
:10658000076FADEC33F000C104F101C105F102C1A8
:1065900006F103C107F118C100F119C101F11AC1D7
:1065A00002F11BC103F107B2DAEF32F0A1EC33F0D4
:1065B000DCEF32F09CEC33F000C118F101C119F1AD
:1065C00002C11AF103C11BF1120097EC34F059C15A
:1065D00000F15AC101F1060EBDEC0BF0E8CF04F159
:1065E000070EBDEC0BF0E8CF05F1080EBDEC0BF08B
:1065F000E8CF06F1090EBDEC0BF0E8CF07F19CECFB
:1066000033F000C124F101C125F102C126F103C11B
:1066100027F1290E046F000E056F000E066F000EA5
:10662000076FADEC33F0EE0E046F430E056F000EF6
:10663000066F000E076FA1EC33F024C104F125C1F1
:1066400005F126C106F127C107F1ADEC33F000C119
:106650001CF101C11DF102C11EF103C11FF1120E97
:10666000BDEC0BF0E8CF04F1130EBDEC0BF0E8CF5E
:1066700005F1140EBDEC0BF0E8CF06F1150EBDECE4
:106680000BF0E8CF07F10D0E006F000E016F000E4A
:10669000026F000E036FADEC33F0180E046F000EA6
:1066A000056F000E066F000E076FCDEC33F01CC1B6
:1066B00004F11DC105F11EC106F11FC107F1A1ECD6
:1066C00033F06A0E046F2A0E056F000E066F000E7F
:1066D000076F9CEC33F01200BF0EFA6E200E3A6F7B
:1066E000396BD8900037013702370337D8B07DEFC8
:1066F00033F03A2F72EF33F039073A070353D8B427
:1067000012000331070B80093F6F03390F0B010F94
:10671000396F80EC5FF0406F390580EC5FF0405DD1
:10672000405F396B3F33D8B0392739333FA992EFF7
:1067300033F04051392712000101BCEC34F0D8B0DD
:106740001200010103510719346F7FEC34F0D89027
:106750000751031934AF800F12000101346BA3EC11
:1067600034F0D8A0B9EC34F0D8B012008EEC34F08C
:1067700097EC34F01F0E366FCFEC34F00B35D8B0F9
:106780007FEC34F0D8A00335D8B01200362FBCEF20
:1067900033F034B1A6EC34F012000101346B045133
:1067A0000511061107110008D8A0A3EC34F0D8A0F9
:1067B000B9EC34F0D8B01200086B096B0A6B0B6BA4
:1067C000CFEC34F01F0E366FCFEC34F007510B5D79
:1067D000D8A4F7EF33F006510A5DD8A4F7EF33F0F1
:1067E0000551095DD8A4F7EF33F00451085DD8A036
:1067F0000AEF34F00451085F0551D8A0053D095F48
:106800000651D8A0063D0A5F0751D8A0073D0B5F8F
:10681000D8900081362FE4EF33F034B1A6EC34F099
:10682000346BA3EC34F0D890D3EC34F007510B5D0B
:10683000D8A427EF34F006510A5DD8A427EF34F02E
:106840000551095DD8A427EF34F00451085DD8A0A4
:1068500036EF34F0003F36EF34F0013F36EF34F0DE
:10686000023F36EF34F0032BD8B4120034B1A6EC5B
:1068700034F012000101346BA3EC34F0D8B01200F4
:10688000D8EC34F0200E366F00370137023703376B
:1068900011EE33F00A0E376FE7360A0EE75CD8B018
:1068A000E76EE552372F4CEF34F0362F44EF34F0DB
:1068B00034B12981D890120001010A0E346F200EE4
:1068C000366F11EE29F03451376F0A0ED890E65228
:1068D000D8B0E726E732372F67EF34F003330233BF
:1068E00001330033362F61EF34F0E750FF0FD8A0AB
:1068F0000335D8B0120029B1A6EC34F012000451CF
:1069000000270551D8B0053D01270651D8B0063DF6
:1069100002270751D8B0073D032712000051086F26
:106920000151096F02510A6F03510B6F12000101EF
:10693000006B016B026B036B12000101046B056BB2
:10694000066B076B12000335D8A012000351800BB1
:10695000001F011F021F031F003FB6EF34F0013F6D
:10696000B6EF34F0023FB6EF34F0032B342B03259F
:1069700012000735D8A012000751800B041F051F15
:10698000061F071F043FCCEF34F0053FCCEF34F077
:10699000063FCCEF34F0072B342B072512000037CD
:1069A000013702370337083709370A370B37120028
:1069B0000101296B2A6B2B6B2C6B2D6B2E6B2F6BB4
:1069C000306B316B326B336B120001012A510F0BAC
:1069D0002A6F2B510F0B2B6F2C510F0B2C6F2D513E
:1069E0000F0B2D6F2E510F0B2E6F2F510F0B2F6F83
:1069F00030510F0B306F31510F0B316F32510F0B84
:106A0000326F33510F0B336F1200899C000EC76E2B
:106A1000200EC66E9E96C69EC50EC96EFF0E9EB611
:106A200002D0E82EFCD79E96C69E000EC96EFF0EC1
:106A30009EB602D0E82EFCD7C9CF00F69E96C69E21
:106A4000000EC96EFF0E9EB602D0E82EFCD7C9CF4D
:106A500001F6898C1200000EC76E200EC66E899C4E
:106A60009E96C69EC80EC96EFF0E9EB602D0E82E38
:106A7000FCD79E96C69E000EC96EFF0E9EB602D033
:106A8000E82EFCD7C9CF02F69E96C69E000EC96EB0
:106A9000FF0E9EB602D0E82EFCD7C9CF03F69E9615
:106AA000C69E000EC96EFF0E9EB602D0E82EFCD721
:106AB000C9CF0AF69E96C69E000EC96EFF0E9EB600
:106AC00002D0E82EFCD7C9CF0BF69E96C69E000ECC
:106AD000C96EFF0E9EB602D0E82EFCD7C9CF12F6C3
:106AE0009E96C69E000EC96EFF0E9EB602D0E82E80
:106AF000FCD7C9CF13F6898C1200000EC76E200E8A
:106B0000C66E899C9E96C69EE80EC96EFF0E9EB606
:106B100002D0E82EFCD79E96C69E000EC96EFF0ED0
:106B20009EB602D0E82EFCD7C9CF1AF69E96C69E16
:106B3000000EC96EFF0E9EB602D0E82EFCD7C9CF5C
:106B40001BF69E96C69E000EC96EFF0E9EB602D024
:106B5000E82EFCD7C9CF22F69E96C69E000EC96EBF
:106B6000FF0E9EB602D0E82EFCD7C9CF23F69E9624
:106B7000C69E000EC96EFF0E9EB602D0E82EFCD750
:106B8000C9CF2AF69E96C69E000EC96EFF0E9EB60F
:106B900002D0E82EFCD7C9CF2BF6898C1200000E4C
:106BA000C76E200EC66E899C9E96C69E240EC96E28
:106BB000FF0E9EB602D0E82EFCD79E96C69EE40E2F
:106BC000C96EFF0E9EB602D0E82EFCD7898C899C38
:106BD0009E96C69E200EC96EFF0E9EB602D0E82E6F
:106BE000FCD79E96C69E5F0EC96EFF0E9EB602D063
:106BF000E82EFCD7898C899C9E96C69E210EC96E74
:106C0000FF0E9EB602D0E82EFCD79E96C69EC00E02
:106C1000C96EFF0E9EB602D0E82EFCD7898C899CE7
:106C20009E96C69E260EC96EFF0E9EB602D0E82E18
:106C3000FCD79E96C69E000EC96EFF0E9EB602D071
:106C4000E82EFCD7898C120010A806D08994000E7B
:106C5000C76E220EC66E05D08984000EC76E220E46
:106C6000C66E050EE82EFED7120010A802D0898449
:106C700001D08994050EE82EFED7120024EC36F0E0
:106C80009E96C69E000EC96EFF0E9EB602D0E82EDE
:106C9000FCD79E96C69E000EC96EFF0E9EB602D011
:106CA000E82EFCD7C9CFABF59E96C69E000EC96EE6
:106CB000FF0E9EB602D0E82EFCD7C9CFACF59E964B
:106CC000C69E000EC96EFF0E9EB602D0E82EFCD7FF
:106CD000C9CFADF59E96C69E000EC96EFF0E9EB63C
:106CE00002D0E82EFCD7C9CFAEF59E96C69E000E08
:106CF000C96EFF0E9EB602D0E82EFCD7C9CFAFF505
:106D00009E96C69E000EC96EFF0E9EB602D0E82E5D
:106D1000FCD7C9CFB0F59E96C69E000EC96EFF0E79
:106D20009EB602D0E82EFCD7C9CFB1F535EC36F0CF
:106D3000120024EC36F09E96C69E800EC96EFF0EA1
:106D40009EB602D0E82EFCD79E96C69EABC5C9FF64
:106D5000FF0E9EB602D0E82EFCD79E96C69EACC50E
:106D6000C9FFFF0E9EB602D0E82EFCD79E96C69EA7
:106D7000ADC5C9FFFF0E9EB602D0E82EFCD79E9689
:106D8000C69EAEC5C9FFFF0E9EB602D0E82EFCD748
:106D90009E96C69EAFC5C9FFFF0E9EB602D0E82ED6
:106DA000FCD79E96C69EB0C5C9FFFF0E9EB602D008
:106DB000E82EFCD79E96C69EB1C5C9FFFF0E9EB6B3
:106DC00002D0E82EFCD735EC36F0120024EC36F079
:106DD0009E96C69E070EC96EFF0E9EB602D0E82E86
:106DE000FCD79E96C69E000EC96EFF0E9EB602D0C0
:106DF000E82EFCD7C9CFABF59E96C69E000EC96E95
:106E0000FF0E9EB602D0E82EFCD7C9CFACF59E96F9
:106E1000C69E000EC96EFF0E9EB602D0E82EFCD7AD
:106E2000C9CFADF59E96C69E000EC96EFF0E9EB6EA
:106E300002D0E82EFCD7C9CFAEF535EC36F024EC05
:106E400036F09E96C69E21C0C9FFFF0E9EB602D0A8
:106E5000E82EFCD79E96C69E000EC96EFF0E9EB60B
:106E600002D0E82EFCD7C9CFB2F535EC36F01200CF
:106E700024EC36F09E96C69E870EC96EFF0E9EB617
:106E800002D0E82EFCD79E96C69EABC5C9FFFF0E6A
:106E90009EB602D0E82EFCD79E96C69EACC5C9FF12
:106EA000FF0E9EB602D0E82EFCD79E96C69EADC5BC
:106EB000C9FFFF0E9EB602D0E82EFCD79E96C69E56
:106EC000AEC5C9FFFF0E9EB602D0E82EFCD735EC4A
:106ED00036F024EC36F09E96C69E22C0C9FFFF0E07
:106EE0009EB602D0E82EFCD79E96C69EB2C5C9FFBC
:106EF000FF0E9EB602D0E82EFCD735EC36F012001D
:106F000024EC36F09E96C69E870EC96EFF0E9EB686
:106F100002D0E82EFCD79E96C69E000EC96EFF0ECC
:106F20009EB602D0E82EFCD79E96C69E800EC96EF5
:106F3000FF0E9EB602D0E82EFCD79E96C69E800E0F
:106F4000C96EFF0E9EB602D0E82EFCD79E96C69E56
:106F5000800EC96EFF0E9EB602D0E82EFCD735EC2F
:106F600036F0120024EC36F09E96C69E870EC96E4F
:106F7000FF0E9EB602D0E82EFCD79E96C69E000E4F
:106F8000C96EFF0E9EB602D0E82EFCD79E96C69E16
:106F9000000EC96EFF0E9EB602D0E82EFCD79E965C
:106FA000C69E800EC96EFF0E9EB602D0E82EFCD79C
:106FB0009E96C69E800EC96EFF0E9EB602D0E82E2B
:106FC000FCD735EC36F0120010A82DD024EC36F0AA
:106FD0009E96C69E22C0C9FFFF0E9EB602D0E82E26
:106FE000FCD79E96C69E450EC96EFF0E9EB602D079
:106FF000E82EFCD735EC36F024EC36F09E96C69E93
:107000008F0EC96EFF0E9EB602D0E82EFCD79E965C
:10701000C69E000EC96EFF0E9EB602D0E82EFCD7AB
:1070200035EC36F0120024EC36F09E96C69E22C057
:10703000C9FFFF0E9EB602D0E82EFCD79E96C69ED4
:10704000010EC96EFF0E9EB602D0E82EFCD735ECBD
:1070500036F024EC36F09E96C69E910EC96EFF0E59
:107060009EB602D0E82EFCD79E96C69EA50EC96E8F
:10707000FF0E9EB602D0E82EFCD735EC36F012009B
:1070800024EC36F09E96C69E22C0C9FFFF0E9EB627
:1070900002D0E82EFCD79E96C69E810EC96EFF0ECA
:1070A0009EB602D0E82EFCD735EC36F0120024EC68
:1070B00036F09E96C69E22C0C9FFFF0E9EB602D035
:1070C000E82EFCD79E96C69E010EC96EFF0E9EB698
:1070D00002D0E82EFCD735EC36F0120024EC36F066
:1070E0009E96C69E910EC96EFF0E9EB602D0E82EE9
:1070F000FCD79E96C69EA50EC96EFF0E9EB602D008
:10710000E82EFCD735EC36F0120024EC36F09E96D3
:10711000C69E910EC96EFF0E9EB602D0E82EFCD719
:107120009E96C69E000EC96EFF0E9EB602D0E82E39
:10713000FCD735EC36F012000501256B266B276B6A
:10714000286B899A400EC76E200EC66E9E96C69E0C
:10715000030EC96EFF0E9EB602D0E82EFCD79E9697
:10716000C69E27C5C9FFFF0E9EB602D0E82EFCD7EB
:107170009E96C69E26C5C9FFFF0E9EB602D0E82E7B
:10718000FCD79E96C69E25C5C9FFFF0E9EB602D0AF
:10719000E82EFCD79E96C69EC952FF0E9EB602D020
:1071A000E82EFCD7898A0F01C950FF0A01E11200BD
:1071B00005012E51130A05E005012E51170A0CE0B6
:1071C00012000501E00E256FFF0E266F0F0E276FD0
:1071D000000E286FF5EF38F00501E00E256FFF0E69
:1071E000266FFF0E276F000E286F899A400EC76E1C
:1071F000200EC66E9E96C69E030EC96EFF0E9EB6EC
:1072000002D0E82EFCD79E96C69E27C5C9FFFF0E6A
:107210009EB602D0E82EFCD79E96C69E26C5C9FF14
:10722000FF0E9EB602D0E82EFCD79E96C69E25C5C0
:10723000C9FFFF0E9EB602D0E82EFCD79E96C69ED2
:10724000C952FF0E9EB602D0E82EFCD7898A0F01E4
:10725000C950FF0A1DE005012E51130A05E0050182
:107260002E51170A0BE012000501000E256F000ECB
:10727000266F100E276F000E286F12000501000EFA
:10728000256F000E266F000E276F010E286F12006B
:107290000501256B266B276B286B05012E51130A00
:1072A00005E005012E51170A0CE012000501000E41
:1072B000216F000E226F080E236F000E246F6AEFFD
:1072C00039F00501000E216F000E226F800E236F32
:1072D000000E246F21C500F122C501F123C502F182
:1072E00024C503F125C504F126C505F127C506F11E
:1072F00028C507F10DEC32F000C125F501C126F5D6
:1073000002C127F503C128F5899A400EC76E200EE9
:10731000C66E9E96C69E030EC96EFF0E9EB602D026
:10732000E82EFCD79E96C69E27C5C9FFFF0E9EB6C7
:1073300002D0E82EFCD79E96C69E26C5C9FFFF0E3A
:107340009EB602D0E82EFCD79E96C69E25C5C9FFE4
:10735000FF0E9EB602D0E82EFCD79E96C69EC9525E
:10736000FF0E9EB602D0E82EFCD7898AC950FF0ACC
:1073700008E104C125F505C126F506C127F507C1B9
:1073800028F5D890050124332333223321332151AA
:10739000E00B216F2167D4EF39F02267D4EF39F089
:1073A0002367D4EF39F024676AEF39F00501200E26
:1073B0002527E86A2623E86A2723E86A282312009B
:1073C000E86A05012E51130A06E005012E51170A3D
:1073D0000BE0020E120005012851000A03E12751BB
:1073E000F00B07E0010E120005012851000A01E030
:1073F000010E120029C500F12AC501F12BC502F1C9
:107400002CC503F125C504F126C505F127C506F1F4
:1074100028C507F19CEC33F003BF1200E0EC39F013
:10742000D8A472EF3AF0899A400EC76E200EC66E4D
:107430009E96C69E060EC96EFF0E9EB602D0E82E20
:10744000FCD7898A899A9E96C69E020EC96EFF0E47
:107450009EB602D0E82EFCD79E96C69E27C5C9FFD1
:10746000FF0E9EB602D0E82EFCD79E96C69E26C57D
:10747000C9FFFF0E9EB602D0E82EFCD79E96C69E90
:1074800025C5C9FFFF0E9EB602D0E82EFCD79E96FA
:10749000C69E000EC96EFF0E9EB602D0E82EFCD727
:1074A000898A899A9E96C69E050EC96EFF0E9EB663
:1074B00002D0E82EFCD79E96C69EC952FF0E9EB6FD
:1074C00002D0E82EFCD7C9B05BEF3AF0898A0501FB
:1074D000200E2527E86A2623E86A2723E86A28235E
:1074E000FAEF39F01200899A400EC76E200EC66E70
:1074F0009E96C69E060EC96EFF0E9EB602D0E82E60
:10750000FCD7898A899A9E96C69EC70EC96EFF0EC1
:107510009EB602D0E82EFCD7898A0501256B266B22
:10752000276B286B1200899A400EC76E200EC66E1C
:107530009E96C69E050EC96EFF0E9EB602D0E82E20
:10754000FCD79E96C69EC952FF0E9EB602D0E82E6C
:10755000FCD7C9CF33F5898A1200899A400EC76ECD
:10756000200EC66E9E96C69EB90EC96EFF0E9EB6C2
:1075700002D0E82EFCD7898A1200899A400EC76E85
:10758000200EC66E9E96C69EAB0EC96EFF0E9EB6B0
:1075900002D0E82EFCD7898AFF0EE82EFED7120013
:1075A000E0EC39F0D8A41200899A400EC76E200E84
:1075B000C66E9E96C69E030EC96EFF0E9EB602D084
:1075C000E82EFCD79E96C69E27C5C9FFFF0E9EB625
:1075D00002D0E82EFCD79E96C69E26C5C9FFFF0E98
:1075E0009EB602D0E82EFCD79E96C69E25C5C9FF42
:1075F000FF0E9EB602D0E82EFCD79E96C69EC952BC
:10760000FF0E9EB602D0E82EFCD7898A0F01C95022
:10761000FF0AD8A4C7EF3DF00501FE0E336F3EEC24
:1076200036F0ABC534F5ACC535F5ADC536F5AEC5F0
:1076300037F5AFC538F5B0C539F5B1C53AF50784AA
:10764000B6C166F1B7C167F1B8C168F1B9C169F1F6
:107650004BC14FF14CC150F14DC151F14EC152F1EE
:1076600057C159F158C15AF1B7EC27F000C13BF5A9
:1076700001C13CF502C13DF503C13EF505015D6761
:1076800049EF3BF05E6749EF3BF05F6749EF3BF046
:1076900060674DEF3BF05AEF3BF05DC504F15EC50E
:1076A00005F15FC506F160C507F19CEC33F003BF3F
:1076B000C7EF3DF059C13FF55AC140F5B5C541F599
:1076C000B6C542F514EC31F036C645F537C646F579
:1076D0000601406773EF3BF0416773EF3BF0426791
:1076E00073EF3BF0436777EF3BF088EF3BF097ECAD
:1076F00034F09DEC34F036C600F137C601F140C6D7
:1077000004F141C605F19CEC33F003AFC7EF3DF047
:107710000101036B026B1AC600F11BC601F101AF38
:1077200096EF3BF0FF0E026FFF0E036F0101076B38
:10773000066B1CC604F11DC605F105AFA4EF3BF0B6
:10774000FF0E066FFF0E076FA1EC33F00101076B10
:10775000066B1EC604F11FC605F105AFB4EF3BF082
:10776000FF0E066FFF0E076FA1EC33F00101076BF0
:10777000066B20C604F121C605F105AFC4EF3BF04E
:10778000FF0E066FFF0E076FA1EC33F0D8900101DA
:107790000333023301330033D89001010333023342
:1077A0000133003300C147F501C148F50101036B06
:1077B000026B22C600F123C601F101AFE4EF3BF0FA
:1077C000FF0E026FFF0E036F0101076B066B24C6ED
:1077D00004F125C605F105AFF2EF3BF0FF0E066F91
:1077E000FF0E076FA1EC33F00101076B066B26C695
:1077F00004F127C605F105AF02EF3CF0FF0E066F5E
:10780000FF0E076FA1EC33F00101076B066B28C672
:1078100004F129C605F105AF12EF3CF0FF0E066F2B
:10782000FF0E076FA1EC33F0D89001010333023350
:1078300001330033D89001010333023301330033A5
:1078400000C149F501C14AF50101036B026B2AC66B
:1078500000F12BC601F101AF32EF3CF0FF0E026FD9
:10786000FF0E036F0101076B066B2CC604F12DC6DA
:1078700005F105AF40EF3CF0FF0E066FFF0E076FFE
:10788000A1EC33F00101076B066B2EC604F12FC685
:1078900005F105AF50EF3CF0FF0E066FFF0E076FCE
:1078A000A1EC33F00101076B066B30C604F131C661
:1078B00005F105AF60EF3CF0FF0E066FFF0E076F9E
:1078C000A1EC33F0D89001010333023301330033CC
:1078D000D8900101033302330133003300C14BF56B
:1078E00001C14CF50101036B026B02C600F103C636
:1078F00001F101AF80EF3CF0FF0E026FFF0E036F4E
:107900000101076B066B04C604F105C605F105AF5E
:107910008EEF3CF0FF0E066FFF0E076FA1EC33F009
:107920000101076B066B06C604F107C605F105AF3A
:107930009EEF3CF0FF0E066FFF0E076FA1EC33F0D9
:107940000101076B066B08C604F109C605F105AF16
:10795000AEEF3CF0FF0E066FFF0E076FA1EC33F0A9
:10796000D89001010333023301330033D890010171
:10797000033302330133003300C14DF501C14EF52D
:107980000101036B026B0AC600F10BC601F101AFE6
:10799000CEEF3CF0FF0E026FFF0E036F0101076B8D
:1079A000066B0CC604F10DC605F105AFDCEF3CF02B
:1079B000FF0E066FFF0E076FA1EC33F00101076B9E
:1079C000066B0EC604F10FC605F105AFECEF3CF0F7
:1079D000FF0E066FFF0E076FA1EC33F00101076B7E
:1079E000066B10C604F111C605F105AFFCEF3CF0C3
:1079F000FF0E066FFF0E076FA1EC33F0D890010168
:107A00000333023301330033D890010103330233CF
:107A10000133003300C14FF501C150F50101036B83
:107A2000026B12C600F113C601F101AF1CEF3DF06D
:107A3000FF0E026FFF0E036F0101076B066B14C68A
:107A400004F115C605F105AF2AEF3DF0FF0E066FF4
:107A5000FF0E076FA1EC33F00101076B066B16C632
:107A600004F117C605F105AF3AEF3DF0FF0E066FC2
:107A7000FF0E076FA1EC33F00101076B066B18C610
:107A800004F119C605F105AF4AEF3DF0FF0E066F90
:107A9000FF0E076FA1EC33F0D890010103330233DE
:107AA00001330033D8900101033302330133003333
:107AB00000C151F501C152F507940501210E326F45
:107AC000899A400EC76E200EC66E9E96C69E060E02
:107AD000C96EFF0E9EB602D0E82EFCD7898A899A1D
:107AE0009E96C69E020EC96EFF0E9EB602D0E82E6E
:107AF000FCD79E96C69E27C5C9FFFF0E9EB602D034
:107B0000E82EFCD79E96C69E26C5C9FFFF0E9EB6E0
:107B100002D0E82EFCD79E96C69E25C5C9FFFF0E53
:107B20009EB602D0E82EFCD725EE33F0322F02D0DD
:107B3000A5EF3DF09E96C69EDECFC9FFFF0E9EB616
:107B400002D0E82EFCD796EF3DF0898A899A9E965E
:107B5000C69E050EC96EFF0E9EB602D0E82EFCD75B
:107B60009E96C69EC952FF0E9EB602D0E82EFCD746
:107B7000C9B0B0EF3DF0898A0501200E2527E86ADB
:107B80002623E86A2723E86A282388EC32F01200CB
:107B900021C500F122C501F123C502F124C503F17D
:107BA000899A400EC76E200EC66E9E96C69E0B0E1C
:107BB000C96EFF0E9EB602D0E82EFCD79E96C69EDA
:107BC00002C1C9FFFF0E9EB602D0E82EFCD79E96DA
:107BD000C69E01C1C9FFFF0E9EB602D0E82EFCD79B
:107BE0009E96C69E00C1C9FFFF0E9EB602D0E82E2B
:107BF000FCD79E96C69EC952FF0E9EB602D0E82EB6
:107C0000FCD725EE33F00501200E326F9E96C69EFE
:107C1000C952FF0E9EB602D0E82EFCD7C9CFDEFFB8
:107C2000322F06EF3EF0898A1200899A400EC76E05
:107C3000200EC66E9E96C69E900EC96EFF0E9EB614
:107C400002D0E82EFCD79E96C69E000EC96EFF0E8F
:107C50009EB602D0E82EFCD79E96C69E000EC96E38
:107C6000FF0E9EB602D0E82EFCD79E96C69E000E52
:107C7000C96EFF0E9EB602D0E82EFCD79E96C69E19
:107C8000C952FF0E9EB602D0E82EFCD7C9CF2DF503
:107C90009E96C69EC952FF0E9EB602D0E82EFCD715
:107CA000C9CF2EF5898A120088EC32F0B5C5E8FFFD
:107CB000D70802E388EC32F0B5C5E8FFC80802E354
:107CC00088EC32F0B5C5E8FFB90802E388EC32F081
:107CD000B5C5E8FFAA0802E388EC32F0B5C5E8FFB5
:107CE0009B0802E388EC32F0E6EC36F0ADEC3AF0BB
:107CF000F29CF29E8B94C69AC290898C9482948C4A
:107D0000720ED36ED3A4FED789968A909390FF0EFD
:107D1000E8CF00F0E82EFED7002EFCD78150F29479
:107D2000F29A9E909D909E929D92F298F292F2907D
:087D3000F286F28E0300FF0051
:10BF0000E844F926000C160C2B0C3F0C520C640C68
:10BF1000760C860C960CA50CB30CC10CCF0CDC0C6B
:06BF2000E80CF40C000C1B
:00000001FF
